:040000000C94320327
:040040000C94BC0B55
:140054004E2557256025722569257B2584258D2596259F2585
:14006800A825B125BA25E125E425E625E925EB25F525F72594
:14007C00FA25FC25FE25002602260426293D001818181800CF
:140090001B00001B1B1B1B001B000000000000001B00060891
:1400A400080611150A001414161D0605060006051615161042
:1400B8001C000A141E28323C46505A646F797E83888D9297CB
:1400CC009CA1A6ABB0B5B9BDC1C5C9CCCFD2D4D6D8D9DADBEB
:1400E000DCDDDEDFE0E1E2E3E4E5E6E7E8E9EAEBECEDEEEF1E
:1400F400F0F1F2F3F4F5F645161E26252E363D3E4645161EF1
:1401080026252E363D3E4600202020202020202020303030C3
:14011C0030302020202020202020202020202020202020202F
:14013000904040404040404040404040404040400C0C0C0C3B
:140144000C0C0C0C0C0C404040404040400909090909090168
:14015800010101010101010101010101010101010101014040
:14016C0040404040400A0A0A0A0A0A020202020202020202F1
:14018000020202020202020202020240404040200000000035
:14019400000000000000000000000000000000000000000057
:1401A800000000000000000000000000000000000000000043
:1401BC0000000000000000000000000000000000000000002F
:1401D00000000000000000000000000000000000000000001B
:1401E400000000000000000000000000000000000000000007
:1401F8000000000000000000000000000000000000000000F3
:14020C000000000000E06735000000200303000000A000009C
:140220000000010000000001000000000001010000000000C6
:14023400060008020000140008000002000000000001010086
:1402480040771B0080EE360010936B0070E9D700406F4001FE
:14025C00A0C5AC010F2A103A371A2D2F30133A371A3D413FC1
:1402700035003A0039003B0035000804000000000000000254
:14028400000200000000000600FAFFF9FF020005000200F96B
:14029800FFFAFF06000000000002000400000001000000004D
:1402AC0000000C001000140019002000280032003C005000EF
:1402C00064007800A000C800FA0040019001F000E900E10060
:1402D400D400C700B400A000820064004600000001000000FA
:1402E800F000E900E100D400C700B400A0008200640046002D
:1402FC00320028001E0016000F000F2A103A371A2D2F3013DE
:140310003A371A3D413F41463D5043204154543D4B42442003
:14032400200050432F4B4244203F2856464F3D4E4F2900534A
:14033800544F524544202020202020202020200053503346D7
:14034C0048492C535033565A580044696769526558202076C0
:140360002E302E393762002532640038313720454D55005079
:1403740043204D4F4445004F5054494F4E0044524D206D6F35
:140388006465202020202020200046696C7465722F6D756CD5
:14039C0074692020200046696C7465722062616E64207365FD
:1403B0007400546F6E652067656E657261746F72200053775E
:1403C4006565702020202020202020202000536D6172742084
:1403D80074756E65207365742000444453206F706572617443
:1403EC00696F6E20200041474320434F4E4649472020202056
:14040000200049462073657474696E672020202020005043E8
:14041400206D6F6E69746F7220202020200044445320736539
:140428007474696E67202020200046696C7465722073776941
:14043C00746368202000412F442073657474696E67202020FB
:1404500020004F5054494F4E5300546F6E65200078202533A6
:140464006400534554204D554C5449504C4945520041474342
:14047800202533640041474320434F4E46494700256C6448B6
:14048C007A200046494C54455220535749544348004D554C1C
:1404A0005449202020004455414C202020200046494C544531
:1404B40052204D4F44452020202020002564200046494C5425
:1404C80045522054554E450054554E452049462046524551F4
:1404DC0020200044524D202856464F3D45584954290053457E
:1404F000542033362737373727323136487A0053455420338E
:140504002732323227373834487A00505245434953494F4EEE
:140518002032304D487A00256C64200053455420324D487ADC
:14052C00002564204D487A200044445320434C4B2046524511
:140540005100414439383530200041443938353120004444D7
:14055400532054595045002020202020005357454550002595
:140568003564204F4E3A25356400446F6E652E2E2E00532DA1
:14057C004D6574657220636F6E6669672E2E002A0025356494
:140590002025356400412F44200042414E4B310042414E4B3C
:1405A40032003F25356400564F4C003E0044414C00204F465F
:1405B800462020200044415300204D414E55414C00414153FE
:1405CC000041474300540044002E002000002E20002A2000D2
:1405E0002B00256400530025356400204C4F434B0041004276
:1405F400004D454D253264200025386C7500253464200053CB
:140608005049204D4F4E49544F52003C696E746567657220B3
:14061C006F6E6C79207072696E742C20757365202D6C667093
:140630003F3F20746F2072656C696E6B3E00286E756C6C204F
:140644007074722070617373656429006162636465660030FE
:14065800006162636465660030000100CFE5D8E0CDBFDEBF73
:14066C00C659D0400AEA08830024E4EBF4E016E0E03BF107FC
:1406800011F00192FBCF0083E0E1F2E0A0E6B0E016E0E436CC
:14069400F10721F0C89531960D92F9CF0E94032EFFCF0E947B
:1406A800333A41E050E002C04F5F5F4F40175107DCF30E9442
:1406BC00363A08950E9424390E944A3A249741E050E060E0AC
:1406D00070E0FE01408351836283738312C041E050E060E0F2
:1406E40070E0FE012080318042805380240E351E461E571E6F
:1406F800FE012082318242825382FE0120843184428453840C
:14070C00FE0160807180828093806214730484049504FCF2F8
:1407200024960E94273A249608950E94333A402F2090CA00B9
:140734002094E091C000F091C1003080322030822090CB005B
:140748002094E091C800F091C90030803220308244FF02C0AD
:14075C00AC9A01C0AC9845FF02C0AD9A01C0AD9846FF02C0E4
:14077000979A01C0979847FF02C0DF9A01C0DF9800002090EB
:14078400CA00E091C000F091C1003080322830820AE010E08E
:1407980086DF2090CA002094E091C000F091C1003080322045
:1407AC00308240FF02C0AC9A01C0AC9841FF02C0AD9A01C031
:1407C000AD9842FF02C0979A01C0979843FF02C0DF9A01C07E
:1407D400DF9800002090CA00E091C000F091C10030803228A3
:1407E80030820AE010E05BDF2090CA002094E091C000F09157
:1407FC00C10030803220308200ED17E04EDF0E94363A0895B4
:140810000E94333A402F2090CB00E091C800F091C9003080A8
:14082400322830822090CA002094E091C000F091C100308063
:140838003220308244FF02C0AC9A01C0AC9845FF02C0AD9A0B
:14084C0001C0AD9846FF02C0979A01C0979847FF02C0DF9AE9
:1408600001C0DF9800002090CA00E091C000F091C1003080AF
:14087400322830820AE010E014DF2090CA002094E091C00038
:14088800F091C10030803220308240FF02C0AC9A01C0AC981A
:14089C0041FF02C0AD9A01C0AD9842FF02C0979A01C09798D5
:1408B00043FF02C0DF9A01C0DF9800002090CA00E091C000D4
:1408C400F091C1003080322830820AE010E0E9DE2090CA0007
:1408D8002094E091C000F091C10030803220308200ED17E04D
:1408EC00DCDE0E94363A08950E944A3A00EA16E821E030E070
:14090000DFDE2090CA002094E091C000F091C1003080322083
:1409140030822090CB002094E091C800F091C9003080322069
:14092800308200E41CE920E030E0C6DE08E2F9DE0CE0F7DEEA
:14093C0006E0F5DE01E0F3DE00E117E220E030E0B9DE0E9419
:14095000273A08950E944A3A422F602F77276130E0E07E07FB
:1409640069F06230E0E07E0771F06330E0E07E0779F0643019
:14097800E0E07E0781F013C0042F00580150D1DE0EC0042F56
:14098C0000540150CCDE09C0042F0C560150C7DE04C0042FBD
:1409A0000C520150C2DE0E94273A08950E94333A402F042FA3
:1409B4002DDF0AE010E075DE0E94363A08950E944E3AA22E4D
:1409C800602F4E815F812A2D062FC0DF04C0FA010191AF01B1
:1409DC00E7DFFA0120802220C1F70E942A3A08950E944A3AE3
:1409F000B901A801042F99DE442706C0FB01049107DF6F5F70
:140A04007F4F43954830C0F300E88DDE0E94273A08952AE808
:140A180030E008E410E0E6DF22E930E000E510E0E1DF2AE956
:140A2C0030E008E510E0DCDF22EA30E000E610E0D7DF2AEA52
:140A400030E008E610E0D2DF22EB30E000E710E0CDDF0895C6
:140A5400002311F4A89801C0A89A0895023011F0013011F41D
:140A6800A99A01C0A998023021F480916800813031F0013072
:140A7C0031F480916800823011F400936800209068000215E7
:140A900009F441C00230F9F42090F8043090F904442437FC31
:140AA4004094552447FC5094809091069090920660908F06E6
:140AB80070909006620C731C841C951C7092900660928F0627
:140ACC0090929206809291061EC02090F8043090F904442404
:140AE00037FC4094552447FC5094809091069090920660900C
:140AF4008F067090900662187308840895087092900660921B
:140B08008F0690929206809291060093680008950E944E3A1F
:140B1C00AE98DF98AA98AE9A0AE010E0BEDDAA980AE010E0ED
:140B3000BADDDF9A0AE010E0B6DDDF986091E904442712C0A2
:140B4400862F8078A82E803811F4AA9A01C0AA980AE010E03C
:140B5800A6DDDF9A0AE010E0A2DDDF98660F4395483060F3A5
:140B6C006091E804442712C0862F8078A82E803811F4AA9AD7
:140B800001C0AA980AE010E08EDDDF9A0AE010E08ADDDF98E8
:140B9400660F4395483060F30AE010E082DDAE980E942A3AB0
:140BA80008950E94333AA80124E030E08A010E944039402FBB
:140BBC008AEB90E0E42FFF27E80FF91F44912090E804421530
:140BD00019F04093E804A0DF0E94363A08950E94333AA80163
:140BE4004093E90497DF0E94363A089522242092E9048EEBBA
:140BF8008093E8048DDF08950E944E3A20908C062220C9F07A
:140C0C004090F6045090F7042090F4043090F5048090910627
:140C20009090920660908F06709090062614370448045904CF
:140C340010F4AF98A9C0AF9AA7C0A090B40440E853EC69ECA4
:140C480071E0409091065090920620908F0630909006241693
:140C5C0035064606570608F4AA2440E458E76DE771E04090FE
:140C700091065090920620908F063090900624163506460605
:140C8400570610F4AA24A39440E05DE261E371E0409091069B
:140C98005090920620908F0630909006241635064606570617
:140CAC0010F482E0A82E40E05BE167EB70E0409091065090B3
:140CC000920620908F0630909006241635064606570610F4CB
:140CD40083E0A82E40E454E569E870E04090910650909206F6
:140CE80020908F0630909006241635064606570610F484E0D7
:140CFC00A82E40E85DE86BE570E04090910650909206209072
:140D10008F0630909006241635064606570610F485E0A82E87
:140D240040EC56EC6DE270E0409091065090920620908F068A
:140D380030909006241635064606570610F486E0A82E40E4CF
:140D4C0052E46FE070E0409091065090920620908F063090DA
:140D60009006241635064606570610F487E0A82E2090B40422
:140D7400A21451F0F894A8BAAF9808EC10E091DCAF9A789499
:140D8800A092B4040E942A3A0895DA9A0AE010E086DCDA98A8
:140D9C00D99A0AE010E081DCD9980AE010E07DDC08950E94B6
:140DB000333A44270BC0DA98802F8170813011F4DB9A01C08E
:140DC400DB98DA9A06954395483098F3DA980E94363A08959D
:140DD8000E9424390E944E3AAA242AC0DA9841E050E060E023
:140DEC0070E0FE012680378040845184242235224622572230
:140E000041E050E060E070E0241635064606570611F4DB9A65
:140E140001C0DB98DA9AFE0126803780408451845694479468
:140E280037942794FE012682378240865186A3948A2D803293
:140E3C0098F2DA980E942A3A249608950E944A3A2C97D998EF
:140E5000DA989498D5DE4090FD045090FE042090FB0430901B
:140E6400FC04809091069090920660908F0670909006620C92
:140E7800731C841C951CFE01608671868286938640900505AF
:140E8C0050900605209003053090040530922506209224061D
:140EA000509227064092260640E05DE261E371E0FE0120849A
:140EB400318442845384241635064606570608F0E2C0FE0121
:140EC800208431844284538440E05DE261E371E04219530975
:140EDC0064097509FE014083518362837383FE012080318056
:140EF00042805380120144245524FE01248235824682578268
:140F040040900105509002052090FF0430900005FE016480C1
:140F18007580868097805A924A923A922A92830194010E94A8
:140F2C00F73918012901569447943794279480902606909097
:140F400027066090240670902506621873088408950870920B
:140F54002506609224069092270680922606FE01248035805D
:140F680046805780210122243324FE01608071808280938034
:140F7C006218730884089508FE01608271828282938288E0EE
:140F900090E0FE0120803180428053808A93810192010E9424
:140FA400CB3AFE0104831583268337834090220650902306B2
:140FB8002090200630902106FE0164807580868097805A9287
:140FCC004A923A922A92830194010E94F739409026065090E6
:140FE00027062090240630902506201A310A420A530A30922B
:140FF400250620922406509227064092260688E090E0FE01FE
:1410080024803580468057808A93810192010E94BF3AFE0112
:14101C002080318042805380201A310A420A530AFE0120821B
:1410300031824282538240901E0650901F0620901C063090D5
:141044001D06FE0160807180828093805A924A923A922A9240
:14105800830194010E94F739409026065090270620902406B6
:14106C0030902506201A310A420A530A30922506209224069E
:141080005092270640922606E1C040E05DE261E371E0FE01BB
:141094002084318442845384241A350A460A570AFE01208283
:1410A800318242825382FE0120803180428053801201442488
:1410BC005524FE0124823582468257824090010550900205ED
:1410D0002090FF0430900005FE0164807580868097805A92B3
:1410E4004A923A922A92830194010E94F7391801290156947C
:1410F8004794379427948090260690902706609024067090E0
:14110C002506620C731C841C951C70922506609224069092EB
:14112000270680922606FE01248035804680578021012224F3
:141134003324FE01608071808280938062187308840895084D
:14114800FE01608271828282938288E090E0FE01208031807E
:14115C00428053808A93810192010E94CB3AFE0104831583F3
:1411700026833783409022065090230620902006309021064A
:14118400FE0164807580868097805A924A923A922A9283018E
:1411980094010E94F739409026065090270620902406309039
:1411AC002506200E311E421E531E309225062092240650920B
:1411C00027064092260688E090E0FE01248035804680578023
:1411D4008A93810192010E94BF3AFE01208031804280538055
:1411E800201A310A420A530AFE012082318242825382409018
:1411FC001E0650901F0620901C0630901D06FE016080718031
:14121000828093805A924A923A922A92830194010E94F7397A
:1412240040902606509027062090240630902506200E311E6B
:14123800421E531E30922506209224065092270640922606FB
:14124C0020912606309127060091240610912506BDDD009111
:141260007D00A5DDD99A0AE010E01DDAD9982C960E94273A01
:1412740008950E944E3AA02E44276627CC99FECFF894DD98A6
:14128800CE99FECF0FC0A7FE02C0DD9A01C0DD98AA0CCC9920
:14129C00FECF660FCE9B01C06395CC9BFECF4395483078F3EB
:1412B000CE9BFECFDD9A789404E610E0F4D9062F0E942A3A8F
:1412C40008950E94333A2C9701E02DDA87E594E099838883B8
:1412D80021E001E072DB15C004E4C9DF402F242E332439829B
:1412EC00288222E534E08E010E5F1F4F0E94333DCE01029646
:141300009983888321E002E05CDBEACF2C960E94363A08956E
:141314000E94333AA80181E090E09093E7048093E6044030C1
:14132800E0E05E0754F4409550954F5F5F4F8FEF9FEF9093FF
:14133C00E7048093E6048091D0009091D10001969093D10057
:141350008093D00084EF91E02090D0003090D1008215930582
:141364000CF0A8C08091CC009091CD00803DE7E09E070CF021
:141378009FC0222433243092D1002092D0002090CE00309012
:14138C00CF00281639065CF48101080F191F22E030E00E942C
:1413A00040391093CF000093CE002090CE003090CF00409010
:1413B400CC005090CD004214530474F420908400309085001E
:1413C8004090CE005090CF00421853085092CF004092CE00BE
:1413DC008091CE009091CF008436E0E09E0734F484E690E00D
:1413F0009093CF008093CE002091CE003091CF0008E010E02F
:141404000E94E739209086003090870002151305C4F42090FE
:14141800CE003090CF00220C331C220C331C220C331C30922A
:14142C00E5042092E404910100E410E00E94E7391093E50475
:141440000093E4040CC0209186003091870000E410E00E945C
:14145400E7391093E5040093E4042091CE003091CF000091BD
:14146800E4041091E5040E945C391093E5040093E4041801A7
:14147C003694279436942794369427943092D4002092D300B2
:14149000220C331C220C331C220C331C280142185308509211
:1414A400D6004092D500222433243092CD002092CC000BC042
:1414B8002090CC003090CD002416350624F45093CD00409307
:1414CC00CC002091D5003091D6008A010E94E73926E030E0C0
:1414E0000E94293918012091D3003091D4008A010E94E73975
:1414F400A801559547955595479555954795420D531D440FD7
:14150800551F8091E6049091E7048030E0E09E0724F4409552
:14151C0050954F5F5F4F8A010E94363A08950E94333AA80188
:1415300080ED97E0841795075CF4405D574023E030E08A016A
:141544000E944039A8014053584F0EC04033E8EF5E0754F4D0
:141558004053584F23E030E08A010E944039A801405D5740AF
:14156C008A010E94363A08950E944A3AA80166E011C082E0E9
:14158000869F8CEC94E0F001E80FF91F208031808EEC94E007
:14159400F001E80FF91F318220826A952224261660F3509337
:1415A800CF044093CE0480919400813029F54091D8045091B5
:1415BC00D904440F551F440F551F2090D8043090D904420D38
:1415D000531D2090D6043090D7042A01420C531C420C531CCD
:1415E4002090DA043090DB04420C531C420C531C2AE030E032
:1415F80082010E944039A80120909400222059F5CA018095E4
:14160C0090958F5F9F4F841B950BAC012091D2043091D304BE
:1416200005E010E00E94E739400F511F2091D4043091D5043D
:1416340005E010E00E94E739400F511F2090D8043090D90423
:141648002A0142185308421853082CE030E082010E9440393F
:14165C00A801809194008430C1F5409550954F5F5F4F2090FC
:14167000D0043090D1042A01420C531C420C531CA201209104
:14168400D2043091D30405E010E00E94E739400F511F2091DD
:14169800D4043091D50405E010E00E94E739400F511F2090C6
:1416AC00D6043090D7042A01420C531C420C531CA2012090BD
:1416C000D8043090D904421953092CE030E08A010E94403924
:1416D400A80180919400823081F5CA01809590958F5F9F4FAB
:1416E800841B950B2090D2043090D3042C01420C531C420C5A
:1416FC00531C2090D4043090D504420C531C420C531C420C82
:14171000531C2090D6043090D704420C531C420C531C209007
:14172400DA043090DB04421853084218530828E030E082012F
:141738000E944039A8018A010E94273A089580EE8BBB8EEA82
:14174C008ABB222428BA8FEF87BB80E885BB8FEF84BB88E08F
:1417600082BB80EC81BB0895222426B827B880E888B98EEECB
:1417740086B908950E94913A0E944A3A24B033243092B6044B
:141788002092B50425B03324322C22244090B5045090B604EF
:14179C00422853285092B6044092B50481E02090EF002826DF
:1417B0002092EF00222009F06AC02090EE043090EF044090FA
:1417C400F5005090F600420C531C5092B8044092B70412014B
:1417D800359427943092B8042092B7042224332440907800A9
:1417EC005090790024143504ACF4C201019790937900809375
:14180000780083FF07C084E690E09093B8048093B70406C0C6
:1418140082E390E09093B8048093B70420907A0030907B00D9
:14182800222039F4332029F42090B7043090B80428BA209054
:14183C00EE043090EF043092F6002092F50080916B009091F7
:141850006C00019690936C0080936B0041E050E060E070E093
:14186400409070005090710020906E0030906F00240E351E0D
:14187800461E571E30926F0020926E0050927100409270009D
:14188C00D3C020907A0030907B00222041F4332031F42090B1
:1418A000EE043090EF0428BA0FC02224332440907A00509017
:1418B4007B002414350434F4C201019790937B0080937A0086
:1418C8008091B5049091B6048A30E0E09E074CF082EF93E028
:1418DC002090B5043090B604821593055CF48AE08093F20027
:1418F00020908100222021F081E080938000A8982090F0008C
:141904003090F1000091B5041091B604021913092091F3009E
:141918003091F4000E94E7391093EF040093EE04180130924E
:14192C00ED042092EC042090F80081E082198093F800809154
:14194000F9008F5F8093F9008CE195E0E091F900FF27E80F37
:14195400F91F208033242801420C531C5092EF044092EE04F1
:141968002090D7003090D800440C551C440C551C440C551C09
:14197C00241435047CF42090EE043090EF04220C331C220C76
:14199000331C220C331C3092D8002092D7000FC022243324E8
:1419A4004090D7005090D8002414350434F4C20101979093B9
:1419B800D8008093D70020908300222049F00091EE04109187
:1419CC00EF04D2DD1093EF040093EE040091EE041091EF0433
:1419E000A4DD1093EF040093EE0420907E00222029F090DC62
:1419F4001093EF040093EE042090EE043090EF043092EB04BE
:141A08002092EA04C1018150984F9093EF048093EE041C0178
:141A1C00359427943594279435942794359427943092EF04F1
:141A30002092EE0480916D008033D1F0803CC1F080B3807379
:141A44008093B90480916D0080732090B904281669F0209099
:141A58006D00220C220C20926D002090B90430906D0032289E
:141A6C0030926D000E94273A0E94A83A1895F89464DE74DEE3
:141A8000222425BE2BBE29BEB3D808950E94333A0030E0E032
:141A94001E0724F4009510950F5F1F4FF9012080318020166A
:141AA800310614F411830083442701C0439582E0849FF0015A
:141ABC008EEF90E0E80FF91F20803180F90140805180241406
:141AD000350484F38AE090E020803180821593052CF48081D7
:141AE40091810A9791838083042F0E94363A08950E94243943
:141AF8000E94563AE22E6C97CC2409C0CE010496EC2DFF2734
:141B0C00E80FF91F81E48083C3948C2D8431A0F3409091068F
:141B20005090920620908F0630909006FE01208E318E428E62
:141B3400538E80916800833001F4809168008230C1F420900B
:141B4800F8043090F904442437FC4094552447FC5094FE01C2
:141B5C00608C718C828C938C6218730884089508FE01608E54
:141B7000718E828E938E80916800813001F52090F8043090A5
:141B8400F904442437FC4094552447FC5094FE01608C718C59
:141B9800828C938C621873088408950840E253E060E070E009
:141BAC00640E751E861E971EFE01608E718E828E938EFE01AB
:141BC000208C318C428C538C288239824A825B822DE434E0C8
:141BD4008E010C5F1F4F0E94333D80E1C82E01C0CA94CE013E
:141BE8000496EC2DFF27E80FF91F80818134B1F3AA24A394A2
:141BFC0010C0CE010496EC2DFF27E80FF91F2080CE01069643
:141C1000EC2DFF27E80FF91F2082CA94A3948A2D853068F374
:141C2400CE010696EC2DFF27E80FF91F8EE28083AA24A3947B
:141C380010C0CE010496EC2DFF27E80FF91F2080CE01059607
:141C4C00EC2DFF27E80FF91F2082CA94A3948A2D843068F339
:141C6000CE010596EC2DFF27E80FF91F8EE28083CE010496DC
:141C7400998388832E2D0EA10E94E1046C960E94303A2496DC
:141C880008950E94333A402F2B97242E33243982288225E454
:141C9C0034E08E010E5F1F4F0E94333DCE0102969983888316
:141CB00021E001E00E94E104409091065090920620908F0693
:141CC40030909006FE01278230864186528684E090E09983C9
:141CD80088832FE836E086E0849F800100501F4F0E94383BE3
:141CEC0027E001E001DFFE01278030844184528430929006CF
:141D000020928F0650929206409291062B960E94363A089535
:141D1400269721E001E0ECDE409091065090920620908F062E
:141D2800309090063092FB002092FA005092FD004092FC003B
:141D3C0020908200222049F083E494E0998388832BE001E0F8
:141D50000E94E10408C081E494E0998388832BE001E00E94A2
:141D6400E10420907C00222049F08BE394E0998388832CE0CA
:141D780001E00E94E10414C020908D0630908E06398228821F
:141D8C0027E334E008E015E00E94333D88E095E09983888332
:141DA0002CE001E00E94E104269608950E94563A680166273A
:141DB40044278EE090E08C159D050CF46C01AA2427C02A2C17
:141DC80033242C143D040CF4439563956230E9F4E42EFF24BB
:141DDC00EE2011F4FF2051F0C7018130E0E09E0749F08230B7
:141DF000E0E09E0749F00BC003E00E94D60407C001E00E94CD
:141E0400D60403C002E00E94D60466274427A3948A2D8E302B
:141E1800B0F20E94303A08950E944A3A259720908C0030908D
:141E2C008D00222029F4332019F44FEF50E009C024E030E00B
:141E400000918E0010918F000E944039A801662701C0639535
:141E540082E0869FF0018EE191E0E80FF91F2080318042156B
:141E6800530514F46A3088F3462F552720908000222041F05D
:141E7C00415050404030E0E05E0714F44427552785E394E0D1
:141E90009983888321E002E00E94E1044A30E0E05E0754F4C6
:141EA4005983488322E334E08E010E5F1F4F0E94333D07C027
:141EB80020E334E08E010E5F1F4F0E94333D8A010E5F1F4F1D
:141ECC006FDFCE0102969983888322E002E00E94E104222475
:141EE0003090F200231470F48DE294E09983888329E002E0AC
:141EF4000E94E1048091F20081508093F20008C08AE294E0D2
:141F08009983888329E002E00E94E10425960E94273A0895D1
:141F1C000E94333A62972BE002E00E94AA04409168005527B7
:141F30004130E0E05E0749F04230E0E05E0749F04330E0E0CB
:141F44005E0749F00BC004E00E94D60407C005E00E94D60498
:141F580003C006E00E94D60440919400405D80918300813009
:141F6C0061F489E294E0998388832CE002E00E94E104042F5E
:141F80000E94D60408C087E294E0998388832CE002E00E9475
:141F9400E1042224332440908C0050908D00241435044CF43D
:141FA80081E494E0998388832DE002E00E94E10408C085E280
:141FBC0094E0998388832DE002E00E94E10480917E008130C0
:141FD00049F483E294E0998388832EE002E00E94E10408C081
:141FE40085E294E0998388832EE002E00E94E104209081003F
:141FF800222049F081E294E0998388832FE002E00E94E104E4
:14200C0008C085E294E0998388832FE002E00E94E1042090CE
:142020008000222049F081E494E09983888320E102E00E942C
:14203400E10408C085E294E09983888320E102E00E94E1047F
:1420480062960E94363A08950E94333A0027112722273327CC
:14205C004091F80055272090F800332442155305D1F3209009
:14207000EC043090ED04021513050CF481012F5F3F4F243694
:14208400E0E03E074CF30E94363A08950E94333A80EA9FE05D
:1420980090937B0080937A0044EF51E01AC080EA9FE09093BF
:1420AC007B0080937A0020908E0030908F0035942794309245
:1420C0008F0020928E00810115950795159507950E94D505B3
:1420D400BDDFBCDFA80188EC90E08417950744F484E02090B1
:1420E8008E0030908F0082159305CCF239C080918E00909161
:1420FC008F00843FE1E09E073CF48C599F4F90938F00809350
:142110008E0009C080918E0090918F00C29690938F008093F8
:142124008E008FEF93E020908E0030908F00821593052CF44C
:1421380082EF90938F0080938E0000918E0010918F001595D6
:14214C000795159507950E94D5057CDF7BDFA80180ED97E0DF
:1421600090937B0080937A00443FE1E05E074CF480918E00B8
:1421740090918F00883EE3E09E070CF4BACF8091CE009091F0
:14218800CF008438E3E09E0734F488539F4F9093CF0080935A
:14219C00CE000E94363A089500B30F700895002720916D009E
:1421B00033272033E0E03E0759F02033E0E03E0744F0203C38
:1421C400E0E03E0709F003C001E001C002E02224201618F43A
:1421D80080EA80936D0008950E944E3AA02E8EE090E02090E6
:1421EC00320130903301821593053CF42090FA043324309292
:1422000035012092340180913201909133018230E0E09E07FD
:1422140034F481E090E090933501809334018A2D823061F55D
:142228002090340130903501442437FC4094552447FC5094B8
:14223C0060908D0670908E06882499245A924A923A922A92BE
:14225000830194010E94F739409091065090920620908F066B
:1422640030909006200E311E421E531E3092900620928F0623
:1422780050929206409291068A2D813061F52090340130900C
:14228C003501442437FC4094552447FC509460908D06709076
:1422A0008E06882499245A924A923A922A92830194010E9422
:1422B400F739409091065090920620908F0630909006201A32
:1422C800310A420A530A3092900620928F0650929206409233
:1422DC009106AA2081F481E090E020903201309033018215D9
:1422F0009305A4F4C101029790933301809332010DC08091D4
:142304003201909133018E30E0E09E072CF40396909333010A
:142318008093320148E55BE160E070E0409091065090920693
:14232C0020908F0630909006241635064606570660F440E070
:142340005AE562E672E05093900640938F0670939206609341
:14235400910640E05AE562E672E04090910650909206209056
:142368008F0630909006421553056405750560F448E55BE127
:14237C0060E070E05093900640938F067093920660939106B7
:142390000E942A3A08950E94333A402F239784E090E099836E
:1423A40088832FE836E086E0849F800100501F4F0E94383B10
:1423B80081E090E0998388839E012E5F3F4F86E0849F800155
:1423CC000C5F1E4F0E94383B2A802092680023960E94363A81
:1423E00008950E94333A402F239722242A8284E090E0998332
:1423F40088832FE836E086E0849F800100501F4F0E945C3B9C
:14240800209068002A8281E090E0998388839E012E5F3F4F4A
:14241C0086E0849F80010C5F1E4F0E945C3B23960E94363AC6
:1424300008950E94523A88E493E06C0184E190E05C0188E5E2
:1424440092E020906B0030906C008215930508F085C0222419
:14245800332430926C0020926B006091D7007091D800759523
:14246C0067957595679575956795AB012090360130903701C9
:142480002B01421853085092370140923601640D751D16012A
:142494002A0C3B1C26163706BCF480E190E020908E003090AF
:1424A8008F008215930574F420908C0030908D0040908E0013
:1424BC0050908F004218530850928F0040928E0016012A18BE
:1424D0003B08621573054CF520908C0030908D0040908E009E
:1424E40050908F00420C531C50928F0040928E006C32E1E088
:1424F8007E07BCF42224332440908C0050908D0024143504C4
:14250C0074F480918E0090918F008C3BE2E09E0734F48C59C9
:142520009F4F90938F0080938E008FEF93E020908E00309077
:142534008F008215930524F490938F0080938E0024E030E056
:1425480000918E0010918F000E9440390E94D505509337017E
:14255C00409336010E942D3A08950E944A3A402F229760917C
:142570008E0070918F00423099F4CB01C29690938F00809351
:142584008E008FEF93E020908E0030908F008215930524F4F0
:1425980090938F0080938E00413099F480918E0090918F008F
:1425AC00C29790938F0080938E008436E0E09E0734F484E6BE
:1425C00090E090938F0080938E008DE194E09983888321E03A
:1425D40002E00E94E10426E430E000918E0010918F000E947F
:1425E8004039E0DB24E030E000918E0010918F000E9440392D
:1425FC000E94D50522960E94273A08950E944E3AA02E229746
:142610008A2D8230B1F480918C0090918D00019690938D0016
:1426240080938C0080E190E020908C0030908D00821593057A
:1426380024F490938D0080938C008A2D813099F480918C0095
:14264C0090918D00019790938D0080938C008030E0E09E07D0
:1426600034F42224332430928D0020928C0089E194E099831A
:14267400888321E002E00E94E10420908C0030908D00222012
:1426880059F4332049F481E194E09983888324E002E00E94DC
:14269C00E10405C000918C0010918D0081DB0AE010E020E0FF
:1426B00030E00E94600322960E942A3A08950E94333A402F28
:1426C40022974230B1F48091840090918500019690938500B8
:1426D800809384008EE090E0209084003090850082159305D1
:1426EC0024F49093850080938400413099F4809184009091CF
:142700008500019790938500809384008130E0E09E0734F42B
:142714002224332430928500209284008DE094E0998388838F
:1427280021E002E00E94E1042090840030908500222071F413
:14273C00332061F485E094E09983888324E002E00E94E10474
:14275000222420927E000BC0009184001091850025DB81E098
:1427640080937E0022242092830022960E94363A08950E944C
:14277800333A402F22974230B1F480918600909187000A96C2
:14278C00909387008093860088E592E020908600309087009A
:1427A0008215930524F49093870080938600413099F480918C
:1427B4008600909187000A9790938700809386008436E0E085
:1427C8009E0734F484E690E0909387008093860081E094E03E
:1427DC009983888321E002E00E94E1042EE130E00091860022
:1427F00010918700045610400E944039D7DA22960E94363A6D
:1428040008950E94333A22972CEB34E00091EC041091ED041D
:14281800159507951595079535D9402F8FEF93E0998388838B
:14282C0021E002E00E94E104042F1127B9DA22243090F20038
:14284000231470F48DE294E09983888329E002E00E94E1046D
:142854008091F20081508093F20008C08AE294E099838883C8
:1428680029E002E00E94E10422960E94363A08950E94333A74
:14287C00402F22974230B1F480918A0090918B000196909308
:142890008B0080938A008CE390E020908A0030908B00821511
:1428A400930524F490938B0080938A00413099F480918A008C
:1428B80090918B00019790938B0080938A008130E0E09E0767
:1428CC0034F481E090E090938B0080938A0020918A003091B8
:1428E0008B0004E010E00E94E7390E94EF058BEF93E0998324
:1428F400888321E002E00E94E10425E030E000918A0010918A
:142908008B000E9440394EDA22243090F200231470F48DE2EB
:14291C0094E09983888329E002E00E94E1048091F2008150C6
:142930008093F20008C08AE294E09983888329E002E00E9432
:14294400E10422960E94363A08950E94563A68012A97AA2409
:14295800BB2482E090E0998388839E012E5F3F4F20906700C2
:14296C0033248601020D131D0E94383BA9C017DCE02E023089
:1429800039F58A819B8101969B838A838AE090E02A803B80ED
:142994008215930520F4C10109969B838A8388EE93E02A80CD
:1429A8003B808215930528F4C101865A9F4F9B838A8380E1F9
:1429BC0097E22A803B808215930520F481E090E09B838A83EA
:1429D0008E2D813031F58A819B8101979B838A838AE090E09D
:1429E4002A803B808215930520F4C10109979B838A8388EE34
:1429F80093E02A803B808215930528F4C1018A5590409B8319
:142A0C008A838A819B818130E0E09E0720F480E197E29B8360
:142A20008A83AA24BB242A803B803982288226EF33E08E0167
:142A34000C5F1F4F0E94333DCE010496998388832BE001E027
:142A48000E94E104ABDB0D3021F580916700803261F488E231
:142A5C008093670080EF93E0998388832CE001E00E94E1046F
:142A70000BC080E2809367008AEE93E0998388832CE001E0AC
:142A84000E94E10400EA16E821E030E00E94600388EB9BE0CB
:142A98005C0184DB0E30B1F408EC10E00E94530388EB9BE0C1
:142AAC005C0182E090E0998388839E012E5F3F4F20906700EF
:142AC00033248601020D131D0E945C3BC501883BEBE09E07B3
:142AD4000CF451CF04C008EC10E00E94530360DB0F30C9F7F4
:142AE8002A960E94303A08950E944E3A249740E457E76BE1DE
:142AFC0070E0409091065090920620908F06309090062416C2
:142B100035064606570678F440909A0050909B002090980034
:142B240030909900FE01208231824282538283E0A82E40E4FA
:142B380057E76BE170E0409091065090920620908F063090CB
:142B4C009006241635064606570600F140EE57E665E370E0CD
:142B60002416350646065706B8F43092990020929800509210
:142B74009B0040929A0040909E0050909F0020909C0030904D
:142B88009D00FE01208231824282538283E0A82E40EE57E60B
:142B9C0065E370E0409091065090920620908F063090900613
:142BB000241635064606570600F140EC5FEC6AE670E02416B1
:142BC400350646065706B8F430929D0020929C0050929F003F
:142BD80040929E004090A2005090A3002090A0003090A100D3
:142BEC00FE01208231824282538283E0A82E40EC5FEC6AE6E8
:142C000070E0409091065090920620908F06309090062416BC
:142C140035064606570600F140E85FE965ED70E02416350650
:142C280046065706B8F43092A1002092A0005092A300409237
:142C3C00A2004090A6005090A7002090A4003090A500FE012D
:142C5000208231824282538282E0A82E40E85FE965ED70E038
:142C6400409091065090920620908F0630909006241635066D
:142C78004606570600F140E45FE660E471E0241635064606EF
:142C8C005706B8F43092A5002092A4005092A7004092A6006D
:142CA0004090AA005090AB002090A8003090A900FE012082B9
:142CB40031824282538282E0A82E40E45FE660E471E04090BA
:142CC80091065090920620908F06309090062416350646068D
:142CDC00570600F140E05FE36BEA71E0241635064606570670
:142CF000B8F43092A9002092A8005092AB004092AA00409086
:142D0400AE005090AF002090AC003090AD00FE012082318261
:142D18004282538282E0A82E40E05FE36BEA71E04090910667
:142D2C005090920620908F0630909006241635064606570662
:142D4000B8F03092AD002092AC005092AF004092AE00409029
:142D54009A0050909B002090980030909900FE012082318261
:142D68004282538283E0A82EFE0120803180428053803092DE
:142D7C00900620928F0650929206409291060A2D0E94300575
:142D900024960E942A3A089524974090910650909206209088
:142DA4008F0630909006FE0120823182428253824090630010
:142DB8005090640020906100309062003092900620928F06F1
:142DCC005092920640929106FE012080318042805380309269
:142DE00062002092610050926400409263002090820081E05C
:142DF4008219809382000091680020906900209268000093DC
:142E08006900249608950E94523A4091F8002090F800421500
:142E1C00E1F366277727CC2419C04091F8002090F800421512
:142E3000E1F3A090EC04B090ED04C5018030E0E09E072CF46E
:142E4400809590958F5F9F4F5C016A157B050CF4B501C394FB
:142E5800C01628F38B010E942D3A08950E944E3A602F2497CF
:142E6C00AA24BB2481E090E0998388839E012D5F3F4F00E410
:142E800010E00E94383B24C0C50101965C0181E090E09983AE
:142E940088839E012E5F3F4F06E010E02F933F9395010E94C3
:142EA800E7393F912F91005C1F4F0E94383B8B818F5F8B837F
:142EBC003A80381609F406C0A5014150504084E690E05C0139
:142ED000C5018331E0E09E07BCF28436E0E09E0721F0AC0184
:142EE4008B818F5F8B83613089F54F5F5F4F83E190E08417F8
:142EF800950714F44427552781E090E0998388839E012D5F18
:142F0C003F4F06E010E02F933F939A010E94E7393F912F91CC
:142F2000005C1F4F0E945C3B84E090E0998388832FE836E072
:142F340006E010E02F933F939A010E94E7393F912F910F5BC8
:142F48001F4F0E945C3B13C084E090E0998388832FE836E0D3
:142F5C0006E010E02F933F939A010E94E7393F912F910F5BA0
:142F70001F4F0E94383B24960E942A3A089501E071DF08959F
:142F840000276EDF0895229782E090E0998388832DE836E04B
:142F98002090670033240091650010916600020D131D0E94D9
:142FAC00383B03E00E943005009180000E942A0581E090E031
:142FC000998388832DE730E007E010E00E94383B84E090E0F2
:142FD4009983888323E035E008E010E00E94383B84E090E0E9
:142FE800998388832FEF34E00CE010E00E94383B84E090E0B7
:142FFC00998388832BEF34E000E110E00E94383B81E090E0B5
:14301000998388832AEF34E005E110E00E94383B82E090E09B
:143024009983888328EF34E006E110E00E94383B84E090E086
:143038009983888324EF34E008E110E00E94383B81E090E077
:14304C00998388832CE836E00CE110E00E94383B89E090E054
:1430600040900105509002052090FF04309000058A93810188
:1430740092010E94CB3A1093210600932006309323062093EC
:14308800220688E090E08A930E94CB3A10931D0600931C06F5
:14309C0030931F0620931E066FDF20918A0030918B0004E0A8
:1430B00010E00E94E7390E94EF05229608950E94563A249782
:1430C400A0907E00BB24002711270E94D505222420927E001A
:1430D80040E050E060E070E0FE014083518362837383C09043
:1430EC00F800DD242090F8003324C214D304D1F3EE24FF2432
:14310000C090F800DD242090F8003324C214D304D1F3209052
:14311400EC043090ED04442437FC4094552447FC5094FE01F8
:143128006080718082809380620C731C841C951CFE0160827E
:14313C00718282829382C70101967C018436E0E09E07C4F2C2
:1431500044E650E060E070E0FE0120803180428053807A938F
:143164006A935A934A93810192010E947C39FE01008311830E
:143178002283338340E058E060E070E0FE01208031804280EE
:14318C005380240E351E461E571E82E090E08A9381019201FA
:1431A0000E9430391093F1000093F00098010FEF17E00E94C9
:1431B40040391093F4000093F300A0927E0024960E94303AFB
:1431C80008950E94563A6C9722243324398E288E3B8E2A8E86
:1431DC0001E00E94950300EA16E821E030E00E94600304C002
:1431F00008EC10E00E9453030E94D2100930C1F3002711271F
:143204000E94D505222420927E0080E092E09093F1008093CB
:14321800F0009C010FEF17E00E9440391093F4000093F300E8
:14322C00EE2485EE93E09983888321E001E00E94E1047FC0C7
:14324000C090EC04D090ED0428E030E086010E944039180116
:1432540004E110E095010E94E7392801420C531C25E130E03D
:1432680082010E94403958011501220C331C220C331C220C1D
:14327C00331C3B822A82D982C8822DED33E08E010C5F1F4F4C
:143290000E94333DCE0104969983888324E001E00E94E1041C
:1432A4009E01285E3F4F84E090E02F933F939C0186010E9435
:1432B80040393F912F910E94460DE02E89E294E099838883F0
:1432CC0021E002E00E94E1040E2D11270E94D60E9E01265E68
:1432E0003F4F86010E94460DE02E89E294E09983888329E0B3
:1432F40002E00E94E1040E2D11270E94D60E22243090F2006C
:14330800231470F48BED93E09983888328E002E00E94E10493
:14331C008091F20081508093F20008C085E294E099838883FA
:1433300028E002E00E94E1040E94D210E02E8E2D8E3009F014
:143344007DCFBBDE6C960E94303A08950E94523AA09701E09F
:143358000E94950300EA16E821E030E00E94600304C008EC71
:14336C0010E00E9453030E94D2100930C1F38AEC93E09983EF
:14338000888321E001E00E94E10440E050E060E070E0FE01E6
:14339400448755876687778740E050E060E070E0FE014087ED
:1433A80051876287738722242092810000270E942A0500E8FD
:1433BC001AE126E030E00E946003CC24DD24A090F800BB24EF
:1433D0002090F8003324A214B304D1F32090EC043090ED0468
:1433E400442437FC4094552447FC5094FE01608471848284E8
:1433F8009384620C731C841C951CFE0160867186828693865F
:14340C00C60101966C018438E3E09E07C4F281E08093800013
:1434200001E00E942A0500E81AE126E030E00E946003CC24F8
:14343400DD24A090F800BB242090F8003324A214B304D1F34C
:143448002090EC043090ED04442437FC4094552447FC509410
:14345C00FE016484758486849784620C731C841C951CFE010A
:143470006486758686869786C60101966C018438E3E09E074B
:14348400C4F2FE01208431844284538444E050E060E070E0A5
:143498005A924A923A922A928A019B010E94F739FE01248430
:1434AC003584468457845A924A923A922A920E947C39109364
:1434C00091000093900001E00E94950382EC93E09983888321
:1434D40021E001E00E94E104FE0120843184428453842C82D8
:1434E8003D824E825F82FE01248435844684578428823982F6
:1434FC004A825B8227EB33E08E01005F1F4F0E94333DCE01B1
:1435100040969983888321E002E00E94E10404C008EC10E098
:143524000E9453030E94D2100E30C1F7A0960E942D3A089545
:143538000E944E3AA29701E00E9495034090FD045090FE044E
:14354C002090FB043090FC04FE01228633864486558640E0D7
:1435600050E060E070E05093FC044093FB047093FE046093EA
:14357400FD0404C008EC10E00E9453030E94D2100930C1F331
:143588005BC10E9424070E948A0E0E94D510A02E0230D1F4C0
:14359C0020908D0630908E0644245524809091069090920644
:1435B00060908F0670909006620C731C841C951C7092900606
:1435C40060928F0690929206809291068A2D8130D1F420902C
:1435D8008D0630908E064424552480909106909092066090C8
:1435EC008F06709090066218730884089508709290066092F8
:143600008F0690929206809291060E94D2100E3091F5809165
:143614006500909166000296909366008093650086E090E047
:1436280020906500309066008215930530F4222433243092A1
:14363C0066002092650082E090E0998388832DE836E0209029
:14365000670033240091650010916600020D131D0E94383B57
:1436640004C008EC10E00E9453030E94D2100E30C1F30E949A
:14367800D210083009F0E0C004C008EC10E00E9453030E9449
:14368C00D2100830C1F381EB93E09983888321E002E00E94D1
:1436A000E104409091065090920620908F0630909006FE01B8
:1436B4002282338244825582ABC00E94D510A02E22242016D0
:1436C800B8F50230C1F448EE53E060E070E04090910650901A
:1436DC00920620908F0630909006240E351E461E571E309287
:1436F000900620928F0650929206409291068A2D8130C1F4E9
:1437040048EE53E060E070E0409091065090920620908F0694
:1437180030909006241A350A460A570A3092900620928F067A
:14372C0050929206409291060E948A0E4AE050E060E070E082
:14374000FE012280338044805580240E351E461E571EFE012B
:14375400228233824482558220908D0630908E0644245524F3
:14376800809091069090920660908F0670909006620C731CD6
:14377C00841C951CFE01228033804480558062147304840486
:143790009504B8F420908D0630908E064424552480909106C1
:1437A4009090920660908F0670909006621873088408950820
:1437B800FE0162827382848295824090910650909206209079
:1437CC008F0630909006FE012682378240865186FE01228060
:1437E0003380448055803092900620928F065092920640929E
:1437F40091060E942407FE0126803780408451843092900610
:1438080020928F0650929206409291060E94D210083009F0CD
:14381C0050CF8BEA93E09983888321E002E00E94E10404C03C
:1438300008EC10E00E9453030E94D2100830C1F30E94D210B4
:14384400013009F0A0CEFE0122843384448455843092FC0419
:143858002092FB045092FE044092FD0404C008EC10E00E94AA
:14386C0053030E94D2100130C1F3A2960E942A3A08950E940C
:14388000523AA09701E00E94950300E513EC20E030E00E94C0
:1438940060034090FD045090FE042090FB043090FC04FE019C
:1438A800248E358E468E578E40E050E060E070E05093FC041B
:1438BC004093FB047093FE046093FD0404C008EC10E00E94E3
:1438D00053030E94D2100930C1F382EA93E09983888321E016
:1438E40001E00E94E10481E080937D008AE993E0998388836A
:1438F80021E002E00E94E1041EC00E94D510A02E023059F4A0
:14390C0081E080937D008AE993E09983888321E002E00E9424
:14392000E1048A2D813059F4222420927D0082E993E099838A
:14393400888321E002E00E94E1040E94D2100E30F1F604C09D
:1439480008EC10E00E9453030E94D2100E30C1F385E893E039
:14395C009983888321E001E00E94E10488E190E06C011FC0A2
:143970000E94D510A02E023019F4C60101966C018A2D81307C
:1439840019F4C60101976C01D982C8822DE733E08E010C5F90
:143998001F4F0E94333DCE0104969983888321E002E00E9486
:1439AC00E1040E94D2100E30E9F680917D00813031F406E037
:1439C00010E096010E94E739680140900105509002052090D4
:1439D400FF0430900005FE01208E318E428E538E40E050E0AA
:1439E80060E070E0509300054093FF0470930205609301057A
:1439FC0040E050E060E070E0509321064093200670932306A8
:143A10006093220640E050E060E070E050931D0640931C06AC
:143A240070931F0660931E0604C008EC10E00E9453030E940D
:143A3800D2100E30C1F301E00E94950384E793E09983888386
:143A4C0021E001E00E94E10440E05DE261E371E05093900690
:143A600040938F0670939206609391064AE050E060E070E0DB
:143A7400409005055090060520900305309004057A936A93EE
:143A88005A934A93810192010E9476391093040500930305B3
:143A9C003093060520930505BCC00E9424070E94D510A02EED
:143AB0000230C1F441E050E060E070E0409005055090060575
:143AC4002090030530900405240E351E461E571E3092040544
:143AD8002092030550920605409205058A2D8130C1F441E019
:143AEC0050E060E070E04090050550900605209003053090C9
:143B00000405241A350A460A570A3092040520920305509213
:143B14000605409205050E94D2100530C1F444E650E060E0AE
:143B280070E040900505509006052090030530900405241AB5
:143B3C00350A460A570A309204052092030550920605409241
:143B500005050E94D2100330C1F444E650E060E070E0409031
:143B64000505509006052090030530900405240E351E461EEE
:143B7800571E309204052092030550920605409205050E94D4
:143B8C00D2100B3059F516014424552443E353E363E373E3CA
:143BA0005A924A923A922A928A019B010E947C391093040597
:143BB4000093030530930605209305054AE050E060E070E0ED
:143BC8003A932A931A930A938A019B010E94F7391093040570
:143BDC000093030530930605209305054090050550900605EA
:143BF0002090030530900405288239824A825B822FE633E00A
:143C04008E010C5F1F4F0E94333DCE0104969983888321E0A1
:143C180002E00E94E1040E94D2100E3009F03FCF409005058C
:143C2C005090060520900305309004054AE050E060E070E02E
:143C40005A924A923A922A928A019B010E94F739109304057B
:143C540000930305309306052093050504C008EC10E00E94EC
:143C680053030E94D2100E30C1F301E00E9495038FE593E07A
:143C7C009983888321E001E00E94E10440E05DE261E371E0B0
:143C90005093900640938F06709392066093910655C00E9463
:143CA40024070E94D510A02E0230C1F441E050E060E070E0C4
:143CB80040900505509006052090030530900405240E351E2D
:143CCC00461E571E30920405209203055092060540920505BD
:143CE0008A2D8130C1F441E050E060E070E040900505509018
:143CF40006052090030530900405241A350A460A570A309240
:143D0800040520920305509206054092050540900505509061
:143D1C0006052090030530900405288239824A825B822FE6E4
:143D300033E08E010C5F1F4F0E94333DCE0104969983888362
:143D440021E002E00E94E1040E94D2100E3009F0A6CF04C00D
:143D580008EC10E00E9453030E94D2100E30C1F38FE493E01F
:143D6C009983888321E001E00E94E10440E05DE261E370E0C0
:143D80005093900640938F067093920660939106FE01208C7E
:143D9400318C428C538C309200052092FF045092020540927A
:143DA800010540E050E060E070E0509321064093200670931B
:143DBC0023066093220640E050E060E070E050931D064093F6
:143DD0001C0670931F0660931E06ADC00E9424070E94D510BD
:143DE400A02E0230C1F441E050E060E070E04090010550907F
:143DF80002052090FF0430900005240E351E461E571E309218
:143E0C0000052092FF0450920205409201058A2D8130C1F40A
:143E200041E050E060E070E040900105509002052090FF043D
:143E340030900005241A350A460A570A309200052092FF040B
:143E480050920205409201050E94D2100530C1F444E650E0DD
:143E5C0060E070E040900105509002052090FF04309000058D
:143E7000241A350A460A570A309200052092FF0450920205AB
:143E8400409201050E94D2100330C1F444E650E060E070E0FC
:143E980040900105509002052090FF0430900005240E351E5C
:143EAC00461E571E309200052092FF045092020540920105EC
:143EC0000E94D2100B30E1F446E950E060E070E04090050591
:143ED4005090060520900305309004057A936A935A934A939A
:143EE800810192010E947639109300050093FF043093020558
:143EFC002093010540900105509002052090FF0430900005C4
:143F1000288239824A825B822FE633E08E010C5F1F4F0E945D
:143F2400333DCE0104969983888321E002E00E94E1040E947D
:143F3800D2100E3009F04ECF04C008EC10E00E9453030E94FD
:143F4C00D2100E30C1F38EE393E09983888321E001E00E94FE
:143F6000E10440E05DE261E372E05093900640938F0670938F
:143F740092066093910655C00E9424070E94D510A02E0230AE
:143F8800C1F441E050E060E070E04090010550900205209022
:143F9C00FF0430900005240E351E461E571E30920005209272
:143FB000FF0450920205409201058A2D8130C1F441E050E0CB
:143FC40060E070E040900105509002052090FF043090000524
:143FD800241A350A460A570A309200052092FF045092020542
:143FEC004092010540900105509002052090FF0430900005B4
:14400000288239824A825B822FE633E08E010C5F1F4F0E946C
:14401400333DCE0104969983888321E002E00E94E1040E948C
:14402800D2100E3009F0A6CF89E090E0409001055090020560
:14403C002090FF04309000058A93810192010E94CB3A10937C
:14405000210600932006309323062093220688E090E08A93C0
:144064000E94CB3A10931D0600931C0630931F0620931E0667
:1440780004C008EC10E00E9453030E94D2100E30C1F381E0BD
:14408C0090E0998388832DE730E007E010E00E945C3B84E0F1
:1440A00090E09983888323E035E008E010E00E945C3B84E0E8
:1440B40090E0998388832FEF34E00CE010E00E945C3BFE011B
:1440C800248C358C468C578C3092FC042092FB045092FE0467
:1440DC004092FD0440EE57E665E370E05093900640938F0619
:1440F0007093920660939106A0960E942D3A08950E944A3A95
:14410400229701E00E94950384E090E0998388832BEF34E0AA
:1441180000E110E00E94383B04C008EC10E00E9453030E946B
:14412C00D2100930C1F38FE293E09983888321E001E00E9421
:14414000E1040E94D2100E30E1F740EE5EE260E070E050930B
:14415400FC044093FB047093FE046093FD0422960E94273AD1
:1441680008950E944E3A2E9701E00E94950384E090E09983AC
:14417C0088832BEF34E000E110E00E94383B04C008EC10E068
:144190000E9453030E94D2100930C1F380E293E099838883B6
:1441A40021E001E00E94E1049DC00E9424070E94D510A02E1F
:1441B8000230C1F445E050E060E070E04090FD045090FE0474
:1441CC002090FB043090FC04240E351E461E571E3092FC0450
:1441E0002092FB045092FE044092FD048A2D8130C1F445E021
:1441F40050E060E070E04090FD045090FE042090FB043090D5
:14420800FC04241A350A460A570A3092FC042092FB0450921F
:14421C00FE044092FD040E94D2100530C1F448EE53E060E0A2
:1442300070E04090FD045090FE042090FB043090FC04241ACA
:14424400350A460A570A3092FC042092FB045092FE0440924D
:14425800FD040E94D2100330C1F448EE53E060E070E040901C
:14426C00FD045090FE042090FB043090FC04240E351E461E03
:14428000571E3092FC042092FB045092FE044092FD040E94E9
:14429400D2100B3061F440EE54E463EA70E05093FC044093EB
:1442A800FB047093FE046093FD044090FD045090FE042090A7
:1442BC00FB043090FC04288239824A825B822FE633E08E016A
:1442D0000C5F1F4F0E94333DCE0104969983888321E002E07C
:1442E4000E94E1040E94D2100E3009F05ECF84E090E0998367
:1442F80088832BEF34E000E110E00E945C3B04C008EC10E0C7
:14430C000E9453030E94D2100E30C1F32E960E942A3A0895C8
:144320000E94523A229701E00E94950302E00E94300504C00A
:1443340008EC10E00E9453030E94D2100930C1F384E193E050
:144348009983888321E001E00E94E104C090F804D090F90428
:14435C006BC00E9424070E94D510A02E023019F4C601019663
:144370006C018A2D813019F4C60101976C010E94D2100530D2
:1443840019F4C60144976C010E94D210033019F4C6014496A4
:144398006C010E94D2100B3019F48CEA9DE06C012090F804CC
:1443AC003090F904442437FC4094552447FC5094809091068A
:1443C0009090920660908F06709090066218730884089508F8
:1443D4007092900660928F069092920680929106D092F904F4
:1443E800C092F8041601442437FC4094552447FC5094620CDF
:1443FC00731C841C951C7092900660928F06909292068092E2
:14441000910616013982288220E133E008E015E00E94333D82
:1444240088E095E09983888321E002E00E94E1040E94D21092
:144438000E3009F090CF82E090E09983888328EF34E006E1CF
:14444C0010E00E945C3B04C008EC10E00E9453030E94D2100F
:144460000E30C1F322960E942D3A08950E94333A629701E00F
:144474000E94950304C008EC10E00E9453030E94D21009309D
:14448800C1F38FEF92E09983888321E001E00E94E10440911B
:14449C008C06442341F026EF32E08E010E5F1F4F0E94333D3F
:1444B00007C02DEE32E08E010E5F1F4F0E94333DCE01029621
:1444C4009983888321E002E00E94E1042BC00E94D510402F72
:1444D800023019F4222420928C06413019F481E080938C0683
:1444EC0022242416D8F420908C06222041F026EF32E08E0105
:144500000E5F1F4F0E94333D07C02DEE32E08E010E5F1F4F5C
:144514000E94333DCE0102969983888321E002E00E94E10489
:144528000E94D2100E3089F681E090E0998388832CE836E01C
:14453C000CE110E00E945C3B04C008EC10E00E9453030E9413
:14455000D2100E30C1F362960E94363A08950E944E3A2897F3
:1445640001E00E94950304C008EC10E00E9453030E94D21004
:144578000930C1F38FED92E09983888321E001E00E94E104C4
:14458C004090F6045090F7042090F4043090F504FE01248270
:1445A0003582468257827EC00E94D510A02E023091F440E441
:1445B40052E46FE070E0FE012480358046805780240E351EA4
:1445C800461E571EFE0124823582468257828A2D813091F41C
:1445DC0040E452E46FE070E0FE012480358046805780241A9F
:1445F000350A460A570AFE01248235824682578240E452E470
:144604006FE070E0FE0124803580468057802416350646064D
:14461800570648F440E452E46FE070E0FE0144835583668375
:14462C00778340E451E86AEB71E0FE01248035804680578088
:14464000421553056405750548F440E451E86AEB71E0FE0196
:1446540044835583668377830E94D2100B3049F440E856E96D
:1446680068E970E0FE014483558366837783FE0124803580C4
:14467C0046805780288239824A825B8228ED32E008E015E07B
:144690000E94333D88E095E09983888321E002E00E94E10496
:1446A4000E94D2100E3009F07DCFFE01248035804680578006
:1446B8003092F5042092F4045092F7044092F60484E090E00C
:1446CC009983888324EF34E008E110E00E945C3B04C008ECC2
:1446E00010E00E9453030E94D2100E30C1F328960E942A3AA4
:1446F40008950E944A3A629701E00E94950304C008EC10E033
:144708000E9453030E94D2100930C1F38DEC92E09983888322
:14471C0021E001E00E94E104442723C00E94D510602F02308A
:1447300009F44395613009F44A9522242616B8F4242E33245C
:144744003982288225EC32E08E010E5F1F4F0E94333DCE018E
:1447580002969983888321E002E00E94E104042F11270E9417
:14476C00D5050E94D2100E30C9F604C008EC10E00E9453033E
:144780000E94D2100E30C1F362960E94273A08950E94333A08
:14479400639701E00E94950304C008EC10E00E9453030E94BA
:1447A800D2100930C1F386EB92E09983888321E001E00E94A0
:1447BC00E1042090FA042A822DC00E94D510402F023019F488
:1447D0008A818F5F8A83413019F48A8181508A838AE02A8054
:1447E400821508F48A838A81813010F481E08A832224241673
:1447F80098F42A8033243982288220EB32E08E010D5F1F4F35
:14480C000E94333DCE0103969983888321E002E00E94E1048D
:144820000E94D2100E3079F62A802092FA0481E090E099830C
:1448340088839E012E5F3F4F05E110E00E945C3B04C008ECE4
:1448480010E00E9453030E94D2100E30C1F363960E94363AF3
:14485C0008950E944E3A669701E00E94950304C008EC10E0C1
:144870000E9453030E94D2100930C1F381EB93E099838883C5
:1448840021E001E00E94E104409091065090920620908F0693
:1448980030909006FE012282338244825582AA24BB2431C023
:1448AC0041E050E060E070E0409091065090920620908F06F3
:1448C00030909006240E351E461E571E3092900620928F0691
:1448D40050929206409291060E942407C50101965C0180E105
:1448E80097E28A159B0578F4FE0122803380448055803092E9
:1448FC00900620928F065092920640929106AA24BB240E9499
:14491000D2100E3059F6FE01228033804480558030929006DF
:1449240020928F06509292064092910604C008EC10E00E940B
:1449380053030E94D2100E30C1F366960E942A3A08950E945E
:14494C004E3A629701E00E94950304C008EC10E00E9453031B
:144960000E94D2100930C1F38AEA92E09983888321E001E0E3
:144974000E94E10468EC70E0AA24A39424C088EE93E090930F
:144988007B0080937A000E94D510402F023011F46F5F7F4F4A
:14499C00413011F4615070401B01442437FC4094552447FCE9
:1449B0005094810192010E946003A8BA2A2C33248FEF90E0F8
:1449C400A82EA218B3080E94D2100E30C1F604C008EC10E073
:1449D8000E9453030E94D2100E30C1F362960E942A3A0895C2
:1449EC000E94523A229781E090E05C0100E21EE420E030E0AE
:144A00000E94600304C008EC10E00E9453030E94D210002356
:144A1400C1F301E00E94950382EA92E09983888321E001E0D8
:144A28000E94E104FDC00E94D510C02E023019F4C501019625
:144A3C005C018C2D813019F4C50101975C018DE090E08A155B
:144A50009B0514F481E05C01C5018130E0E09E071CF48DE093
:144A640090E05C01C5018130E0E09E070CF488C08DE090E070
:144A78008A159B050CF482C002E010E095010E94E739F80186
:144A8C0082E590E0E80FF91F05901490F001099482E992E08C
:144AA0009983888321E002E00E94E1046BC082E892E099834E
:144AB400888321E002E00E94E10462C082E792E09983888355
:144AC80021E002E00E94E10459C082E692E09983888321E055
:144ADC0002E00E94E10450C082E592E09983888321E002E06A
:144AF0000E94E10447C082E492E09983888321E002E00E94A0
:144B0400E1043EC082E392E09983888321E002E00E94E10452
:144B180035C082E292E09983888321E002E00E94E1042CC041
:144B2C0082E192E09983888321E002E00E94E10423C082E0CA
:144B400092E09983888321E002E00E94E1041AC082EF91E0A2
:144B54009983888321E002E00E94E10411C082EE91E09983EE
:144B6800888321E002E00E94E10408C082ED91E099838883F5
:144B7C0021E002E00E94E1040E94D210093009F04DC0C50132
:144B90008130E0E09E070CF438C08DE090E08A159B050CF4E7
:144BA40032C002E010E095010E94E739F8018CE690E0E80F0F
:144BB800F91F05901490F00109940E94E51821C0CADC1FC005
:144BCC000E943F1C1CC0CBDA1AC02224209297008EEA8ABB31
:144BE0008FEE8BBB0E94630910C085DD0EC00E949C1A0BC0CD
:144BF400CDDD09C032DE07C0A6DE05C08FDB03C033DC01C01D
:144C08007BDA01E00E94950304E610E00E9453038BEC91E06E
:144C1C009983888321E001E00E94E1040E94D2100E3009F039
:144C3000FECE22960E942D3A08950E94563A229705E50E94CF
:144C44003B0984E6809F19820882CC242DC004E00E940717E9
:144C580058017501EF2CFF240E2D0E943B091701322C22245E
:144C6C00A218B3080A2D0E943B09C02E288039804424552472
:144C8000809091069090920660908F0670909006620C731CA9
:144C9400841C951C7092900660928F06909292068092910639
:144CA8000E9424078C2D803F81F622960E94303A08950E9439
:144CBC004E3A05E50E943B09602F05E50E943B09A02E05E575
:144CD0000E943B09402F2A2D062F0E94AA04042F0E94D604F0
:144CE4000E942A3A08950E94563A229701E00E94950383ECA4
:144CF80091E09983888321E001E00E94E104AA2468C1CC994B
:144D0C0005C004E40E943B09E02E01C0EE240E94D2100E305D
:144D200011F482E0A82E0E9419128E2D8A3609F054C10AE6FC
:144D34000E943B09E02ECE2CDD24C6018431E0E09E0709F49E
:144D480040C18531E0E09E0709F43DC185E18C159D053CF16A
:144D5C00C6018130E0E09E0749F18230E0E09E0749F1833028
:144D7000E0E09E0749F18430E0E09E0709F4F8C08530E0E04D
:144D84009E0709F4F7C08630E0E09E0709F4F6C08730E0E07D
:144D98009E0709F4FBC08A30E0E09E0709F40FC118C1C6011E
:144DAC008436E0E09E0709F410C111C12224209280000DC1EE
:144DC00081E08093800009C104E40E943B09202E04E42F925C
:144DD4000E943B092F90402E04E44F922F920E943B092F9089
:144DE8004F90602E04E46F924F922F920E943B092F904F903B
:144DFC006F90802E442D55276627772780E197E2A0E0B0E0F4
:144E10007A936A935A934A938C019D010E94F739A801B9015A
:144E240033244424552480E492E4AFE0B0E05A924A923A92B5
:144E38002A928C019D010E94F73918012901240E351E461E81
:144E4C00571E462D55276627772784E690E0A0E0B0E07A93CC
:144E60006A935A934A938C019D010E94F739200E311E421E9D
:144E7400531E682C772488249924260C371C481C591C309201
:144E8800900620928F06509292064092910640E853EC69EC9A
:144E9C0071E0421553056405750548F048E55BE160E070E0EE
:144EB000241635064606570660F440E157E260E070E05093AF
:144EC400900640938F0670939206609391068091680082308C
:144ED800F1F42090F8043090F904442437FC4094552447FC4D
:144EEC005094809091069090920660908F0670909006620CE6
:144F0000731C841C951C7092900660928F06909292068092D2
:144F1400910680916800813031F52090F8043090F9044424D1
:144F280037FC4094552447FC5094809091069090920660907F
:144F3C008F0670909006620C731C841C951C40E253E060E053
:144F500070E0641A750A860A970A7092900660928F0690928E
:144F64009206809291060E94240735C002E00E94300531C08C
:144F780003E00E9430052DC004E40E943B09202E3324309249
:144F8C008D0020928C0023C004E40E943B09202E332430922E
:144FA0008F0020928E00220C331C220C331C30928F00209231
:144FB4008E00810115950795159507950E94D5050AC039DEF0
:144FC80008C077DE06C001E00E94950302C0AA24A394AA2046
:144FDC0009F495CE22960E94303A089522242AB82BB88EE87F
:144FF00080BD89E189B920BC88E18AB908950E944A3A44270E
:145004000AC080EC94E0E42FFF27E80FF91F00810E94043B44
:1450180043954430A0F36091680077276130E0E07E0789F05F
:14502C006230E0E07E0749F06330E0E07E0709F00BC000279D
:145040000E94043B07C001E00E94043B03C002E00E94043B6C
:145054000E94273A08950E944E3A2090C4043324359427942B
:14506800359427943594279435942794442437FC40945524C0
:14507C0047FC509440E051EE65EF75E05A924A923A922A92A1
:145090008A019B010E94F7391093900600938F063093920657
:1450A400209391068091C40499278F7090701C01442437FC5E
:1450B8004094552447FC509440E856E968E970E05A924A92A0
:1450CC003A922A928A019B010E94F739409091065090920670
:1450E00020908F0630909006200E311E421E531E309290067B
:1450F40020928F0650929206409291062090C50433243594E5
:145108002794359427943594279435942794442437FC4094DD
:14511C00552447FC509440E452E46FE070E05A924A923A9252
:145130002A928A019B010E94F7394090910650909206209027
:145144008F0630909006200E311E421E531E30929006209214
:145158008F0650929206409291068091C50499278F70907032
:14516C001C01442437FC4094552447FC509440EA56E861E05A
:1451800070E05A924A923A922A928A019B010E94F7394090B2
:1451940091065090920620908F0630909006200E311E421E80
:1451A800531E3092900620928F06509292064092910620914F
:1451BC00C604332735952795359527953595279535952795A3
:1451D00000E117E20E94E7391801442437FC4094552447FCEB
:1451E4005094809091069090920660908F0670909006620CEB
:1451F800731C841C951C7092900660928F06909292068092D8
:14520C0091062091C60433272F70307008EE13E00E94E73938
:145220001801442437FC4094552447FC50948090910690908B
:14523400920660908F0670909006620C731C841C951C709263
:14524800900660928F0690929206809291068091C7048295DF
:14525C008F7094E6989F1001442437FC4094552447FC50946E
:14527000620C731C841C951C7092900660928F069092920603
:14528400809291068091C7048F709AE0989F1001442437FC35
:145298004094552447FC5094620C731C841C951C70929006A8
:1452AC0060928F069092920680929106AA240FC084EC94E083
:1452C000EA2DFF27E80FF91F208080EC94E0EA2DFF27E80FDA
:1452D400F91F2082A3948A2D843070F340E853EC69EC71E0FA
:1452E800409091065090920620908F06309090064215530589
:1452FC006405750548F048E55BE160E070E0241635064606C9
:14531000570660F440E157E260E070E05093900640938F060D
:145324007093920660939106809168008230F1F42090F80494
:145338003090F904442437FC4094552447FC509480909106EE
:14534C009090920660908F0670909006620C731C841C951C2C
:145360007092900660928F069092920680929106809168003E
:14537400813031F52090F8043090F904442437FC40945524FD
:1453880047FC5094809091069090920660908F067090900670
:14539C00620C731C841C951C40E253E060E070E0641A750ACD
:1453B000860A970A7092900660928F06909292068092910636
:1453C4000E9424070E942A3A089500270E94043B00270E9494
:1453D800043B089508950E944E3AA090C404BB24AA2011F478
:1453EC00BB2099F0C5018130E0E09E0791F08230E0E09E07D5
:1454000091F08030E0E09E07F4F0C5018C30E0E09E0769F0DE
:1454140018C003E00E94300514C002E00E94300510C001E0B4
:145428000E9430050CC040EE5EE260E070E05093FC04409319
:14543C00FB047093FE046093FD040E9424070E942A3A0895F4
:145450000E944A3A20908C0030908D00222029F4332019F4DA
:145464006FEF70E009C024E030E000918E0010918F000E94B8
:145478004039B801442701C0439582E0849FF00188E391E098
:14548C00E80FF91F208031806215730514F44F3088F320900B
:1454A0008000222029F043958FE0841708F44FE0042F0E943B
:1454B400043B0E94273A08950E944A3A229792DD01E00E9434
:1454C80095038BEB91E09983888321E001E00E94E104B4C04D
:1454DC00662777270E941B3B84EC94E0FB01E80FF91F008327
:1454F0000E9419126F5F7F4F6530E0E07E0784F34091C80451
:1455040055274838E0E05E0709F489C088E890E08417950715
:145518000CF43DC04031E0E05E0709F46EC080E190E0841755
:14552C0095071CF14030450709F44FC04130E0E05E0709F467
:145540004EC04230E0E05E0709F44BC04330E0E05E0709F415
:145554004AC04530E0E05E0709F447C04730E0E05E0709F402
:1455680046C04830E0E05E0709F443C067C04038E0E05E07C8
:14557C0009F445C04238E0E05E0709F444C04538E0E05E07D7
:1455900009F443C057C0473EE0E05E0709F44DC087EE90E057
:1455A4008417950784F04B3BE0E05E0709F43BC04C3BE0E05E
:1455B8005E0709F438C04D3BE0E05E0709F435C03DC0473F63
:1455CC00E0E05E0709F435C037C000270E94043B33C03DDDA8
:1455E00031C000270E94043B2DC009DD2BC000270E94043BF8
:1455F40027C0F3DE25C000270E94043B21C000270E94043B15
:145608001DC000270E94043B19C000270E94043B15C00027CC
:14561C000E94043B11C000270E94043B0DC0D1DE0BC0D6DEC5
:1456300009C000270E94043B05C00ADF03C009E80E94043B52
:145644004BCF22960E94273A0895222733278BB380638BBBD6
:145658008EEC8ABB002702C02F5F3F4F2835E2E03E0724F4FE
:14566C0029B2332424FCF6CF2835E2E03E070CF401E08EEF51
:145680008ABBDD9ADC9808950E94333A222733278BB3806376
:145694008BBB8EEC8ABB0027112702C02F5F3F4F203AEFE097
:1456A8003E0724F429B2332424FCF6CFCC9921C0222714C017
:1456BC00CC9BFECF29B2332424FCFCCFCD9B03C040E051E00D
:1456D00002C044275527283020F4040F151F1595079523956C
:1456E400293050F3CC9BFECF29B2332424FCFCCFCC9BFECF91
:1456F80002C0002711278EEF8ABBDD9ADC980E94363A089521
:14570C000E94563AE02E62978BEF90E0FE010AE010E0FA9300
:14572000EA939A938A930E94EB3A0DE00E949503CC2401C00F
:14573400C3948C2D8A3040F4CE01EC2DFF27E80FF91F2080A6
:145748002E14A1F72C2C332444245524FE01228633864486B9
:14575C005586FE0122843384448455843092900620928F06C2
:145770005092920640929106809168008230F1F42090F80486
:145784003090F904442437FC4094552447FC5094809091069E
:145798009090920660908F0670909006620C731C841C951CDC
:1457AC007092900660928F06909292068092910680916800EE
:1457C000813031F52090F8043090F904442437FC40945524AD
:1457D40047FC5094809091069090920660908F067090900620
:1457E800620C731C841C951C40E253E060E070E0641A750A7D
:1457FC00860A970A7092900660928F069092920680929106E6
:1458100021E001E00E947A0DAA24BB24B9C017DFE02E222409
:14582400201608F0B3C0F89404EF11E00E94530329DFE02E51
:145838007894BA2CAA242E2C3324A20CB31CC5018070803008
:14584C00E0EF9E0709F09EC0CC2401C0C3948C2D8A3040F4CE
:14586000CE01EC2DFF27E80FF91F20802E14A1F78C2D8A302A
:1458740008F08CC040E856E968E970E0FE01228433844484B0
:145888005584241635064606570608F07DC0FE012284338484
:14589C00448455844AE050E060E070E05A924A923A922A921D
:1458B0008A019B010E94F739180129016C2C7724882499240C
:1458C400260C371C481C591CFE012286338644865586FE016E
:1458D80022843384448455843092900620928F0650929206A5
:1458EC0040929106809168008230F1F42090F8043090F904C6
:14590000442437FC4094552447FC5094809091069090920625
:1459140060908F0670909006620C731C841C951C709290067E
:1459280060928F06909292068092910680916800813031F531
:14593C002090F8043090F904442437FC4094552447FC5094DF
:14595000809091069090920660908F0670909006620C731CCC
:14596400841C951C40E253E060E070E0641A750A860A970ACB
:145978007092900660928F06909292068092910621E001E0B7
:14598C000E947A0D8E2D8A3509F043CF40EC55E069ED71E051
:1459A000409091065090920620908F063090900642155305CA
:1459B4006405750560F440E853EC69EC71E05093900640934F
:1459C8008F06709392066093910648EE53E060E070E0409048
:1459DC0091065090920620908F06309090062416350646064C
:1459F000570660F440E157E260E070E05093900640938F0627
:145A0400709392066093910662960E94303A08950E94563A96
:145A1800E02E669785E091E0FE0134960AE010E0FA93EA93EC
:145A2C009A938A930E94EB3A0DE00E949503CC2401C0C39426
:145A40008C2D8A3048F4CE010496EC2DFF27E80FF91F20804C
:145A54002E1499F72C2C332444245524FE0126863786408AAA
:145A6800518AFE012684378440885188288239824A825B823C
:145A7C0027EB31E008E015E00E94333D88E095E09983888300
:145A900024E001E00E94E104AA24BB2474C0D7DDE02E2224AD
:145AA400201608F06EC0F89404EF11E00E945303E9DDE02E56
:145AB8007894BA2CAA242E2C3324A20CB31CC5018070803086
:145ACC00E0EF9E0709F059C0CC2401C0C3948C2D8A3048F489
:145AE000CE010496EC2DFF27E80FF91F20802E1499F78C2DD0
:145AF4008A3008F046C04AE050E060E070E0FE012684378498
:145B080040885188241635064606570608F037C0FE01268432
:145B1C003784408851884AE050E060E070E05A924A923A929B
:145B30002A928A019B010E94F739180129016C2C772488248A
:145B44009924260C371C481C591CFE0126863786408A518A25
:145B5800FE012684378440885188288239824A825B8227EB14
:145B6C0031E008E015E00E94333D88E095E09983888324E01D
:145B800001E00E94E1048E2D8A3509F088CF44E150E060E04A
:145B940070E0FE012684378440885188421553056405750516
:145BA80048F444E150E060E070E0FE0146875787608B718B37
:145BBC00FE0126843784408851882092770066960E94303A9F
:145BD00008950E944A3A442711C086E591E0E42FFF27E80FB6
:145BE400F91F6081675E242F2F5F02E00E94AA04062F0E9405
:145BF800D6044395403168F30E94273A0895EF972297002418
:145C0C000BAE0CAE11241EAE0DAEAA240E943D0D0E94D21017
:145C20000F3011F0AA24A3940E94C9060E947A0486EA91E0B9
:145C34009983888321E001E00E94E10422242092070528E9B7
:145C480031E08E010E5F1F4F0E94333D8BE08AAF0AE010E03D
:145C5C0020E030E00E946003B6DF00E81AE126E030E00E94EF
:145C700060030E940B050E94C5170E94240788E293E29093BE
:145C84007B0080937A0078940E945F180E94481081E0809371
:145C980072008D81863431F08F81893419F081E08093070547
:145CAC00AA2009F005DC8FEF9FE3FE01FF9691838083E5C5EB
:145CC00085B7806885BF889585B78F7785BF0CAC03940CAEBC
:145CD4000E94663DFE01FF96208131810E944039202E8CE1BA
:145CE80095E0ECADFF27E80FF91F208281E00BAC80198BAFD8
:145CFC00222433242E143F041CF4C70101977C01C70181300C
:145D1000E0E09E0751F42090960020929500822D813019F4DB
:145D240081E0809372000E94D5100AAF2224002E201618F48F
:145D38008CE291E07C010E941912209007052220C1F048EE49
:145D4C0053E060E070E0409005055090060520900305309043
:145D60000405240E351E461E571E3092040520920305509261
:145D74000605409205052090950033243FAA2EAAC101813064
:145D8800E0E09E07F1F08230E0E09E0709F4B2C08330E0E0C8
:145D9C009E0709F49DC08430E0E09E0709F49CC08530E0E00D
:145DB0009E0709F49FC08630E0E09E0709F496C08730E0E0F9
:145DC4009E07E1F19CC020907C00222011F000240AAE222467
:145DD8000AAC201498F4409070005090710020906E003090D2
:145DEC006F003092740020927300509276004092750081E0D9
:145E0000809372000AAD0E94F0100BAC002049F020907F0071
:145E1400222019F00E94031402C00E94100F2090720022208F
:145E280039F00E9424070E948A0E22242092720081E0809358
:145E3C00960061C022240AAC201410F5802D813029F48091DA
:145E500077008150809377008AAD823029F4809177008F5FF0
:145E64008093770020907700222019F484E18093770084E1D6
:145E780020907700821518F481E08093770081E0809372007B
:145E8C00809172008130F1F4209068002AAE009177000E944F
:145EA000CB11209068000AAC021439F0C22C002D0E94300513
:145EB4000C2D0E943005009177000E94450E0E9424070E945E
:145EC80048102224209272000BAC0020B1F00E94100F13C0F8
:145EDC000AAD0E94BB130FC00AAD0E945F130BC00AAD0E94CD
:145EF000B31207C00AAD0E94041303C00AAD0E943C140E9494
:145F04008E0F40E050E060E070E040907500509076002090C1
:145F1800730030907400241635064606570619F18090700026
:145F2C009090710060906E0070906F006218730884089508E5
:145F400040E553EC60E070E0461557056805790570F440E033
:145F540050E060E070E0509374004093730070937600609370
:145F680075000E94BF1720908100222031F02224209280002C
:145F7C00022D0E942A0520909700222009F4BFC00BAC002035
:145F900009F4BBC05CDB0AAF2224002E201608F0B4C0F894F3
:145FA40004EF11E00E9453036DDB0AAF78940DAC1EAC102C41
:145FB80000241EAE0DAE2AAC3324020C131C1EAE0DAEC00178
:145FCC008932E0EF9E0709F430C08A32E0EF9E0709F458C060
:145FE0008AE290EF8015910544F08DAD9EAD8D30E0EF9E07AD
:145FF40009F454C05EC08DAD9EAD8233E0EF9E0761F08233B6
:14600800E0EF9E070CF453C08DAD9EAD8A33E0EF9E0719F13D
:14601C004CC00E9478150E9424070E94481081E08093950065
:146030008093720040C080917A0090917B008030E0E09E079B
:146044003CF08FEF9FEF90937B0080937A0031C088EE93E00B
:1460580090937B0080937A002AC087E0809395008093960067
:14606C0040E050E060E070E05093740040937300709376002A
:146080006093750081E080937200EE24FF2413C081E0809342
:14609400950080939600809372000BC00E94CC160E94240719
:1460A8000E94481081E080939500809372008DAD9EAD8070E7
:1460BC008030E0EF9E0719F58AAD863181F08E3171F0863267
:1460D00061F0853251F08E3241F0863331F08D3321F08E3316
:1460E40011F0863481F480919600813039F40AAD0BDB0E94B4
:1460F80024070E94481002C00AAD88DC81E080937200AA24DE
:14610C00BB240E94D2100AAF202E332439AE28AE222019F4B2
:14612000332009F4A5C388AD99AD8130E0E09E0709F46AC3F8
:146134008330E0E09E0709F442C28530E0E09E0709F4F8C26D
:146148008730E0E09E0709F4FDC18830E0E09E0709F45FC132
:14615C008930E0E09E0709F416C18B30E0E09E0709F4A2C0BE
:146170008C30E0E09E0709F418C38D30E0E09E0709F4ABC197
:146184008E30E0E09E0791F07EC308EC10E00E945303C50180
:1461980001965C01883BEBE09E0731F488EE93E09093790022
:1461AC00809378000E94D2100E3059F388EB9BE08A159B0519
:1461C000ECF480919500813009F05BC0009165001091660083
:1461D4000E94A71482E090E0998388832DE836E0209067001F
:1461E80033240091650010916600020D131D0E94383B43C0F8
:1461FC0020908300222091F020907C00222071F08091940025
:146210008F5F8093940082E020909400821588F52224209233
:1462240094002DC080919500813049F5809165009091660053
:146238000296909366008093650086E090E02090650030900E
:14624C0066008215930530F4222433243092660020926500A9
:1462600082E090E0998388832DE836E0209067003324009107
:14627400650010916600020D131D0E94383B81E0809395004D
:146288008093960080937200FCC208EC10E00E945303C50174
:14629C0001965C01883BEBE09E0731F488EE93E0909379001D
:1462B000809378000E94D2100B3059F388EB9BE08A159B0517
:1462C4000CF03DC025C00E94D5100AAF013029F480917700D2
:1462D8008150809377008AAD823029F4809177008F5F8093C8
:1462EC00770020907700222019F484E18093770084E12090AD
:146300007700821518F481E080937700009177000E94450E87
:146314000E94D2100B30B9F6009177000E94F11187E891E07B
:146328009983888321E001E00E94E10400EA16E821E030E0D8
:14633C000E94600311C087E0809395008093960040E050E06F
:1463500060E070E0509374004093730070937600609375002B
:1463640081E080937200EE24FF248DC208EC10E00E945303DF
:14637800C50101965C01883BEBE09E0731F488EE93E09093F3
:14638C007900809378000E94D210093059F388EB9BE08A1563
:1463A0009B05E4F481E080937E0086E090E0909385008093EE
:1463B400840088E092E09093870080938600992790938D00C4
:1463C80080938C002224209283000E948E0F0E94481057C255
:1463DC00809195008F5F8093950086E020909500821518F423
:1463F00083E08093950080919500833018F483E0809395001E
:146404008CE291E07C013FC208EC10E00E945303C5010196EE
:146418005C010E94D2100830A9F301E00E94950386E791E0C2
:14642C009983888321E001E00E94E10486E691E099838883C8
:1464400021E002E00E94E10407C008EC10E00E945303C50175
:1464540001965C010E94D2100F30A9F30E94D210013049F4EF
:146468002224209297008EEA8ABB8FEE8BBB0E9475260E9432
:14647C00D2100C3079F481E0809397008FEE8BBB8EE88ABBF8
:1464900007C008EC10E00E945303C50101965C010E94D21017
:1464A4000F30A9F781E080939500809372000E948E0FE9C18E
:1464B80008EC10E00E945303C50101965C01883BEBE09E0707
:1464CC0031F488EE93E090937900809378000E94D2100D30C6
:1464E00059F388EB9BE08A159B059CF42090830081E0821970
:1464F40080938300882341F0222420927E003324309285000E
:14650800209284000E948E0FBCC120907C0081E08219809352
:14651C007C0081E08093950080937200B0C108EC10E00E946A
:146530005303C50101965C01883BEBE09E0731F488EE93E006
:1465440090937900809378000E94D210073059F388EB9BE027
:146558008A159B05ACF4409091065090920620908F0630906C
:14656C00900630926200209261005092640040926300209023
:1465800068002092690006C00E94CC160E9424070E94481073
:1465940081E0809395008093720075C108EC10E00E94530353
:1465A800C50101965C01883BEBE09E0731F488EE93E09093C1
:1465BC007900809378000E94D210033059F388EB9BE08A1537
:1465D0009B050CF094C080916800833089F544E650E060E083
:1465E40070E0409091065090920620908F06309090067A93CC
:1465F8006A935A934A93810192010E94763910939006009396
:14660C008F06309392062093910644E650E060E070E03A9389
:146620002A931A930A938A019B010E94F7391093900600939A
:146634008F06309392062093910665C02090F8043090F9048A
:14664800442437FC4094552447FC50948090910690909206D0
:14665C0060908F067090900662187308840895087092900659
:1466700060928F06909292068092910644E650E060E070E042
:146684007A936A935A934A93830194010E947639109390068B
:1466980000938F06309392062093910644E650E060E070E037
:1466AC003A932A931A930A938A019B010E94F73910939006D4
:1466C00000938F0630939206209391062090F8043090F90490
:1466D400442437FC4094552447FC509438014901620C731C23
:1466E800841C951C7092900660928F069092920680929106CB
:1466FC0006C00E9478150E9424070E94481081E080939500C5
:1467100080937200BAC008EC10E00E945303C50101965C01E0
:14672400883BEBE09E0731F488EE93E09093790080937800F9
:146738000E94D210053059F388EB9BE08A159B057CF480919A
:14674C006800813021F402E00E9430050FC002E00E943005CA
:1467600001E00E94300508C080916800813021F005E0081B62
:146774000E943005209096002092950081E08093720081C086
:1467880008EC10E00E945303C50101965C01883BEBE09E0734
:14679C0031F488EE93E090937900809378000E94D2100C30F4
:1467B00059F388EB9BE08A159B053CF42090810081E08219FF
:1467C4008093810060C02090800081E0821980938000082F17
:1467D8000E942A05209096002092950052C008EC10E00E94B7
:1467EC005303C50101965C01883BEBE09E0731F488EE93E048
:1468000090937900809378000E94D210013059F388EB9BE06E
:146814008A159B05B4F480917A0090917B008030E0E09E074D
:146828003CF08FEF9FEF90937B0080937A0029C088EE93E027
:14683C0090937B0080937A0022C080919500823021F482E06C
:1468500090E07C0106C082E0809395008CE291E07C012224D5
:14686400332430927B0020927A000DC00E94D2100023E1F318
:146878000E94F624209096002092950081E0809372001ACAF9
:14688C00EF96229608950E9424390E94563A69970024112494
:1468A0001D8A0C8AAFC4EDA1FEA18081853259F00081EBA1F9
:1468B400FCA10E945A3A8C899D8901969D8B8C8B9AC400246A
:1468C80011241B8A0A8A8FEF9FEF9F8B8E8B198A088A83E95E
:1468DC0096E09D838C8380E2888F8DA19EA101969EA38DA315
:1468F000CC24DD24EDA1FEA1208033243F862E86822D932D97
:146904008032E0E09E0759F18332E0E09E0799F08032E0E009
:146918009E078CF18E859F858B32E0E09E07A9F08D32E0E0D8
:14692C009E0759F08033E0E09E07E9F022C088899989816082
:14694000998B888B20C0888999898460998B888B1AC08889F3
:1469540099898860998B888B8BE2888F12C08889998988607D
:14696800998B888B80E2888F0AC0888999898061998B888B56
:14697C0004C081E090E0C82ED92ECC2011F4DD2009F006C0C8
:146990008DA19EA101969EA38DA3ACCFEDA1FEA1008111271D
:1469A4000E94E83C00300107B1F00DA11EA10E94963B1B8BBA
:1469B8000A8B05C08DA19EA101969EA38DA3EDA1FEA100814E
:1469CC0011270E94E83C0030010791F716C0EDA1FEA18081F5
:1469E0008A3289F48FA198A5029698A78FA3E82FF92F3297EC
:1469F400208031803B8A2A8A8DA19EA101969EA38DA3EDA1C2
:146A0800FEA180818E3209F03AC08E2F9F2F01969EA38DA394
:146A1C00E82FF92F008111270E94E83C00300107B1F00DA121
:146A30001EA10E94963B1F8B0E8B05C08DA19EA101969EA3D3
:146A44008DA3EDA1FEA1008111270E94E83C0030010791F7A2
:146A580016C0EDA1FEA180818A3289F48FA198A5029698A7A9
:146A6C008FA3E82FF92F3297208031803F8A2E8A8DA19EA19D
:146A800001969EA38DA3EDA1FEA180818C3651F48E2F9F2F3A
:146A940001969EA38DA3888999898260998B888BEDA1FEA16D
:146AA800208033243F862E86822D932D8835E0E09E0709F4DC
:146ABC00D4C088E582159305A4F08E859F858534E0E09E07AD
:146AD00009F48EC38534E0E09E070CF43EC08E859F85833559
:146AE400E0E09E0709F4D5C136C08E859F858F36E0E09E074F
:146AF80009F4B5C08FE690E02E843F8482159305B4F08E85D8
:146B0C009F858336E0E09E0709F498C18436E0E09E0751F17C
:146B20008536E0E09E0709F463C38636E0E09E0709F45EC3DF
:146B340012C08E859F858337E0E09E0709F47CC28537E0E06E
:146B48009E0709F48CC08837E0E09E0709F487C000C0EDA195
:146B5C00FEA10081EBA1FCA10E945A3A8C899D8901969D8BAC
:146B70008C8B43C30888198801FE49C08FA198A5049698A775
:146B84008FA3E82FF92F34972080318042805380EC2FFD2F94
:146B9800208631864286538640E050E060E070E0EC2FFD2FC4
:146BAC0020843184428453842416350646065706ACF4888910
:146BC00099898860998B888B8DE2888FEC2FFD2F0085118598
:146BD400228533850E94633AEC2FFD2F008711872287338746
:146BE8008AE090E09B838A83EC2FFD2F208431844284538457
:146BFC0048825982222D332D0C811D810E94493CF7C08FA1F8
:146C100098A5029698A78FA3E82FF92F3297208031803F8210
:146C24002E82822D932D8030E0E09E077CF48889998988609D
:146C3800998B888B8DE2888F8E819F81809590958F5F9F4F46
:146C4C009F838E838AE090E0998388832E813F810C811D8166
:146C60000E94E93BCBC00888198801FE13C08FA198A50496C5
:146C740098A78FA3E82FF92F34972080318042805380EC2F90
:146C8800FD2F20863186428653860CC08FA198A5029698A7BE
:146C9C008FA3E82FF92F3297208031803F822E82EDA1FEA1BB
:146CB0008081853711F50888198801FE13C08AE090E09B8312
:146CC4008A83EC2FFD2F208431844284538448825982222D7E
:146CD800332D0C811D810E94493C8CC08AE090E099838883A9
:146CEC002E813F810C811D810E94E93B81C0EDA1FEA18081C5
:146D00008F3661F50888198800FE06C080E3EC81FD8181930D
:146D1400FD83EC830888198801FE13C088E090E09B838A8376
:146D2800EC2FFD2F208431844284538448825982222D332DC6
:146D3C000C811D810E94493C5BC088E090E0998388832E8128
:146D50003F810C811D810E94E93B50C00888198800FE0EC071
:146D640080E3EC81FD818193FD83EC83EDA1FEA12080EC8190
:146D7800FD812192FD83EC830888198801FE13C080E190E013
:146D8C009B838A83EC2FFD2F208431844284538448825982E6
:146DA000222D332D0C811D810E94493C0AC080E190E0998327
:146DB40088832E813F810C811D810E94E93BEDA1FEA1808132
:146DC8008835C1F483E996E0E82EF92E0EC0EE2DFF2D008190
:146DDC0011270E94123DEE2DFF2D00838E2D9F2D0196E82E7C
:146DF000F92EEE2DFF2D2080222069F783E996E0E82EF92EC0
:146E04008E899F898F3FEFEF9E0721F4002411241F8A0E8A3B
:146E18000E881F88002019F4112009F41DC103E916E00E946C
:146E2C0018391F830E83202E312E0E881F88001611060CF0BB
:146E40000FC13F8A2E8A0CC18FA198A5029698A78FA3E82F93
:146E5400F92F3297208031802C8681E090E00A881B8880159B
:146E6800910554F41F8A0E8A22242D868C2F9D2F0C96E82EBF
:146E7C00F92EF0C00C85EBA1FCA10E945A3A8C899D89019669
:146E90009D8B8C8BB2C18FA198A5029698A78FA3E82FF92F87
:146EA4003297A080B1808E899F898F3FEFEF9E0721F40024F7
:146EB80011241F8A0E8A0A881B88002011F4112051F00A2D4D
:146ECC001B2D0E94893B4A885B88401A510A5B8A4A8A0E884B
:146EE0001F88002041F4112031F40A2D1B2D0E94893B1F8BBD
:146EF4000E8B0A881B88002011F4112049F00888198803FEFB
:146F080005C08A899B8901979B8B8A8B0888198804FE28C08B
:146F1C0003FE0AC0088DEBA1FCA10E945A3A8C899D890196D0
:146F30009D8B8C8B0888198802FC54C00FC000E3EBA1FCA1F0
:146F44000E945A3A8C899D8901969D8B8C8B8A899B89019723
:146F58009B8B8A8B222433240A881B882014310454F33CC06C
:146F6C000888198802FC17C00FC000E2EBA1FCA10E945A3AFB
:146F80008C899D8901969D8B8C8B8A899B8901979B8B8A8BE2
:146F9400222433240A881B882014310454F30888198803FE35
:146FA8001DC0088DEBA1FCA10E945A3A8C899D8901969D8B0A
:146FBC008C8B12C0EA2DFB2DC895002DEBA1FCA10E945A3AB0
:146FD0008C899D8901969D8B8C8B8A2D9B2D0196A82EB92EC9
:146FE400EA2DFB2DC895002059F02E883F88822D932D019710
:146FF8009F8B8E8B222001F73320F1F60888198802FEF7C0E6
:14700C000FC000E2EBA1FCA10E945A3A8C899D8901969D8B66
:147020008C8B8A899B8901979B8B8A8B222433240A881B8869
:147034002014310454F3DFC08FA198A5029698A78FA3E82F6C
:14704800F92F3297E080F180EE2031F4FF2021F48EE894E021
:14705C00E82EF92E8E899F898F3FEFEF9E0721F400241124E5
:147070001F8A0E8A0A881B88002011F4112051F00E2D1F2D78
:147084000E9418394A885B88401A510A5B8A4A8A0E881F88A5
:14709800002041F4112031F40E2D1F2D0E9418391F8B0E8B7C
:1470AC000A881B88002011F4112049F00888198803FE05C015
:1470C0008A899B8901979B8B8A8B0888198804FE28C003FE96
:1470D4000AC0088DEBA1FCA10E945A3A8C899D8901969D8BF0
:1470E8008C8B0888198802FC53C00FC000E3EBA1FCA10E94BE
:1470FC005A3A8C899D8901969D8B8C8B8A899B8901979B8BE6
:147110008A8B222433240A881B882014310454F33BC0088849
:14712400198802FC17C00FC000E2EBA1FCA10E945A3A8C89BC
:147138009D8901969D8B8C8B8A899B8901979B8B8A8B2224F7
:14714C0033240A881B882014310454F30888198803FE1CC0E5
:14716000088DEBA1FCA10E945A3A8C899D8901969D8B8C8B16
:1471740011C0EE2DFF2D0081EBA1FCA10E945A3A8C899D89D4
:1471880001969D8B8C8B8E2D9F2D0196E82EF92EEE2DFF2D7B
:14719C002080222059F02E883F88822D932D01979F8B8E8BED
:1471B000222009F73320F9F60888198802FE1DC00FC000E288
:1471C400EBA1FCA10E945A3A8C899D8901969D8B8C8B8A8934
:1471D8009B8901979B8B8A8B222433240A881B882014310471
:1471EC0054F305C083E694E0E82EF92E33CF8DA19EA1019663
:147200009EA38DA3EDA1FEA12080222009F04BCB0C891D89B0
:1472140069960E94303A24960895A02FB12FE22FF32F019091
:147228000D920020E1F70895E02FF12FAA27BB27019000208B
:14723C0011F01196FBCF0A2F1B2F08953A932A931A930A93D8
:147250000895222321F0159507952A95FACF08950F92099092
:14726400002031F035952795179507950A94F8CF0F90089566
:147278006894DA92D12E04C0E894DA92D12ED32617FF04C01D
:14728C00109500950F5F1F4F37FF04C0309520952F5F3F4F48
:1472A0000E945D39D7FE04C0109500950F5F1F4FD9900895ED
:1472B400689401C0E894EA92FA928A93EE24FF2480E1000FC3
:1472C800111FEE1CFF1CE216F30618F0E21AF30A03958A95B4
:1472DC00A1F716F40E2D1F2D8991F990E9900895E89401C07F
:1472F00068942FD0CC2408C0E89401C0689429D037FD53D04E
:14730400B7FD5AD0772488249924AA24BB2441D0C1F044D010
:14731800B1F0E8E2000F111F221F331F771C881C991CAA1C72
:14732C00BB1C88169906AA06BB0628F0881A990AAA0ABB0AF2
:147340000395EA9559F726F4082D192D2A2D3B2D13C07A929F
:147354008A929A92AA92BA92CA92EA938A939A93AA93BA93A8
:147368008B859C85AD85BE85C32E0EF0CB260895C7FC17D044
:14737C00B991A99199918991E991C990B990A990999089909E
:14739000799024960895E02FE12BE22BE32B0895E82FE92B8B
:1473A400EA2BEB2B089500951095209530950F5F1F4F2F4FFF
:1473B8003F4F089580959095A095B0958F5F9F4FAF4FBF4FFA
:1473CC0008950A921A928A939A93029FC001129F900D039F2C
:1473E000900D8C01999189911990099008950E946C3A7F92F3
:1473F4000E94853A39F177240E948B3A19F48C019D0120C0E0
:14740800089FB02CA12C289F902C812C189FA00C911C871C3D
:14741C00099FA00C911C871C199F900C811C0A9F900C811CE5
:14743000389F800C299F800C1A9F800C0B9F800C0B2D1A2D97
:14744400292D382D7F900C947A3AE2E00C94373AE4E00C94DF
:14745800373AE8E00C94373AEE270C94373A5A934A93089549
:14746C00E1E049915991E0FD089569917991E1FD0895A99055
:14748000B990E2FD0895C990D990E3FD0895E990F990089555
:147494007A936A930C94333ABA92AA920C944A3ADA92CA9259
:1474A8000C944E3AFA92EA920C94523A0A92C8950A92319618
:1474BC00C895F02DE9910990099400951095209530950F5F70
:1474D0001F4F2F4F3F4F08958A929A92AA92BA92EA938A9327
:1474E4009A93AA93BA9389859A85AB85BC850895B991A9911E
:1474F80099918991E991B990A9909990899024960895EE2792
:14750C00E02BE12BE22BE32B0895EE27E82BE92BEA2BEB2B35
:147520000895FA93EA93BA93AA939A938A933A932A931A93A5
:147534000A939A928A927A926A925A924A923A922A921A925A
:147548000A920FB60A92089509900FBE09901990299039906B
:14755C0049905990699079908990999009911991299139914D
:1475700089919991A991B991E991F99108950F920990002044
:1475840031F0000F111F221F331F0A94F8CF0F9008950F92BE
:147598000990002031F036952795179507950A94F8CF0F9032
:1475AC0008950A921A92002411240030010741F016950795DD
:1475C00010F4020E131E220F331FF5CF002D112D199009907E
:1475D4000895AA93BA93EA93FA930A92AF81B885ED81FE817C
:1475E8000030010731F0C8950D92319601501040F7CF099073
:1475FC00F991E991B991A991249608950E94333A402F20906E
:14761000AE063090AF06222011F4332021F04A3011F40DE026
:14762400F1DF5D9BFECF4CB9042F11270E94363A08955F9BA4
:14763800FECF0CB111270895E199FECF1FBB0EBBE09A0DB3BB
:14764C0008950E94333AE199FECF1FBB0EBB2DBB4FB7F8941A
:14766000E29AE19A4FBF002711270E94363A08950E94523AD5
:14767400C22ED32EA02EB12E688579854C2D5D2D0EC00A2D71
:147688001B2D0E94203BE42FF52F00838A2D9B2D0196A82E03
:14769C00B92E4F5F5F4F262E372E61507040222061F7332090
:1476B00051F70E942D3A08950E94523AC22ED32EA02EB12E0C
:1476C400688579854C2D5D2D0EC0E42FF52F20810A2D1B2D9F
:1476D8000E94273B8A2D9B2D0196A82EB92E4F5F5F4F262E17
:1476EC00372E61507040222061F7332051F70E942D3A0895E9
:14770000822F932F01968E7F800F911F082F192F0895E02FF4
:14771400F12FAA27BB27C895002019F031961196FACF0A2F98
:147728001B2F08950E944E3A602F712F02C06F5F7F4FE62F9A
:14773C00F72F008111270E94043D00300107A9F7AA24BB24F2
:14775000E62FF72F80818D3239F481E090E0A82EB92E6F5FA1
:147764007F4F07C0E62FF72F80818B3211F46F5F7F4F442777
:14777800552712C00AE010E0242F352F0E94D73A402F512F7C
:14778C00E62FF72F21906E2F7F2F3324420D531D4053504079
:1477A000E62FF72F008111270E94E83C0030010729F7AA20F9
:1477B40011F4BB2039F0042F152F009510950F5F1F4F02C069
:1477C800042F152F0E942A3A08950E94563AC22ED32E402F01
:1477DC00512F2B97AD88BE88CC2029F4DD2019F467EA74E024
:1477F00046C022242A866C2F7D2F665F7F4F39C02A2D3B2DF7
:147804000C2D1D2D0E945A39E02EF12E0A30E0E01E0774F404
:14781800862F972F0197282E392E682F792F8E2D9F2DC09670
:14782C00E22DF32D808317C08A2D9B2D8031E0E09E0789F42D
:14784000862F972F0197282E392E682F792F86E994E0EE2D27
:14785400FF2DE80FF91F4080E22DF32D40822A2D3B2D0C2D3C
:147868001D2D0E945C39C02ED12ECC2009F0C4CFDD2009F030
:14787C00C1CF262F372F042F152F0E940F392B960E94303A7F
:1478900008950E9424390E94563A6A97CAA4DBA440E050E0D8
:1478A40060E070E0EC2FFD2F26A037A040A451A4241635060E
:1478B8004606570629F480EB94E0E82EF92E79C02224298EA4
:1478CC008C2F9D2F4996E82EF92E61C02C2C3D2C442437FC88
:1478E0004094552447FC5094EC2FFD2F66A077A080A491A463
:1478F4005A924A923A922A92062D172D282D392D0E947839AB
:14790800A02EB12E0A30E0E01E0774F48E2D9F2D0197282EC2
:14791C00392EE82EF92E8A2D9B2DC096E22DF32D808317C0D5
:147930008C2D9D2D8031E0E09E0789F48E2D9F2D0197282EB8
:14794400392EE82EF92E8FE994E0EA2DFB2DE80FF91F408091
:14795800E22DF32D40822C2C3D2C442437FC4094552447FC3E
:14796C005094EC2FFD2F66A077A080A491A45A924A923A92D2
:147980002A92062D172D282D392D0E947639EC2FFD2F06A3C4
:1479940017A320A731A740E050E060E070E0EC2FFD2F26A099
:1479A80037A040A451A4241635064606570609F08FCF2E2D4B
:1479BC003F2D0CA11DA10E940F396A960E94303A2496089593
:1479D00080E191E0202E312E280E391EE22DF32DC895002DDE
:1479E400112704701070089580E191E0202E312E280E391EBA
:1479F800E22DF32DC895002D112702701070089580E191E029
:147A0C00202E312E280E391EE22DF32DC895002D11270071CA
:147A2000107008950E94333A402F512F042F152F0E94F63CEC
:147A34000030010739F0042F152F015610400F5B1F4F02C025
:147A4800042F152F0E94363A0895E091AC06F091AD06019319
:147A5C00F093AD06E093AC0608950E9424390E94333A229757
:147A70002C803D803092AD062092AC0622E030E00C2F1D2F27
:147A84000A5F1F4F0E94803B402F512F598348832E813F81B5
:147A980008E810E00E9449342224E091AC06F091AD0620829C
:147AAC002C803D800E2F1F2F0219130922960E94363A249617
:147AC00008951093B3040093B20408952091B2043091B304F6
:147AD4000DE61EE40E94D73A802F912F875C9F4C9F77909380
:0C7AE800B3048093B204082F192F0895F6
:00000001FF
